:020000040000FA
:0408000098EF0BF072
:1008100003B275EF05F0F2B493EF05F09EB09BEFD5
:1008200005F09EB2A3EF05F0F2A81AEF04F0F2B2C1
:1008300023EF04F0F2B01FEF04F047EF0BF0F29655
:10084000F29047EF0BF0CD90F2929EA02DEF04F0C6
:100850000101533F2DEF04F0542BB2C1B6F1B3C1E7
:10086000B7F1B4C1B8F1B5C1B9F1AEC1B2F1AFC120
:10087000B3F1B0C1B4F1B1C1B5F1AAC1AEF1ABC130
:10088000AFF1ACC1B0F1ADC1B1F1A6C1AAF1A7C140
:10089000ABF1A8C1ACF1A9C1ADF1A2C1A6F1A3C150
:1008A000A7F1A4C1A8F1A5C1A9F19EC1A2F19FC160
:1008B000A3F1A0C1A4F1A1C1A5F19AC19EF19BC170
:1008C0009FF19CC1A0F19DC1A1F1CECF9AF1CFCFF4
:1008D0009BF153C19CF154C19DF1CF6ACE6A0101D5
:1008E000536B546B9E90CD800FBC0F8E0FBA7CEF74
:1008F00004F00F8A47EF0BF013880F8C0FBEB9EF8F
:1009000004F09AC19EF19BC19FF19CC1A0F19DC1D1
:10091000A1F19EC1A2F19FC1A3F1A0C1A4F1A1C107
:10092000A5F1A2C1A6F1A3C1A7F1A4C1A8F1A5C1D7
:10093000A9F1A6C1AAF1A7C1ABF1A8C1ACF1A9C1A7
:10094000ADF1AAC1AEF1ABC1AFF1ACC1B0F1ADC177
:10095000B1F1AEC1B2F1AFC1B3F1B0C1B4F1B1C147
:10096000B5F1B2C1B6F1B3C1B7F1B4C1B8F1B5C117
:10097000B9F101015E6B5F6B606B616B9A515E2731
:100980009B515F239C5160239D5161239E515E27A3
:100990009F515F23A0516023A1516123A2515E2783
:1009A000A3515F23A4516023A5516123A6515E2763
:1009B000A7515F23A8516023A9516123AA515E2743
:1009C000AB515F23AC516023AD516123AE515E2723
:1009D000AF515F23B0516023B1516123B2515E2703
:1009E000B3515F23B4516023B5516123B6515E27E3
:1009F000B7515F23B8516023B9516123D8900101E9
:100A0000613360335F335E33D8900101613360330B
:100A10005F335E33D8900101613360335F335E33FF
:100A200000C10CF101C10DF102C10EF103C10FF1C2
:100A300004C110F105C111F106C112F107C113F192
:100A400008C114F109C115F10AC116F10BC117F162
:100A500034C135F111B838EF05F00101620E046FB1
:100A6000010E056F000E066F000E076F41EF05F0D7
:100A70000101A70E046F020E056F000E066F000E37
:100A8000076F5EC100F15FC101F160C102F161C198
:100A900003F165EC2FF003BF04D01CBE02D01CA0F4
:100AA000108C11A059EF05F010BA59EF05F00F8026
:100AB000108A0CC100F10DC101F10EC102F10FC18C
:100AC00003F110C104F111C105F112C106F113C106
:100AD00007F114C108F115C109F116C10AF117C1D6
:100AE0000BF135C134F147EF0BF00392ABB2AB9889
:100AF000AB88030103EE00F080517F0BE92604C0B0
:100B0000EFFF802B8151805D700BD8A48B82000099
:100B10008051815D700BD8A48B9281518019D8B41B
:100B2000079047EF0BF0F2940101453F47EF0BF0C0
:100B3000462B47EF0BF09E900101533F47EF0BF020
:100B4000542B47EF0BF09E9211B843EF08F00400CE
:100B500066A1ABEF05F08BB4B5EF05F010ACB5EFC7
:100B600005F08B84109CB6EF05F08B94077C07ACE6
:100B7000D1EF05F0C274C2B4CBEF05F0C3CFB7F527
:100B8000C4CFB8F50501D890B833B733D890B8338F
:100B9000B733D2EF05F0C3CF55F1C4CF56F1D2EF42
:100BA00005F0C28207B444EF06F047C14BF148C1DB
:100BB0004CF149C14DF14AC14EF15EC162F15FC1D4
:100BC00063F160C164F161C165F113A8EAEF05F05A
:100BD000138C13989AC1BAF19BC1BBF19CC1BCF1B3
:100BE0009DC1BDF19EC1BEF19FC1BFF1A0C1C0F1C9
:100BF000A1C1C1F1A2C1C2F1A3C1C3F1A4C1C4F199
:100C0000A5C1C5F1A6C1C6F1A7C1C7F1A8C1C8F168
:100C1000A9C1C9F1AAC1CAF1ABC1CBF1ACC1CCF138
:100C2000ADC1CDF1AEC1CEF1AFC1CFF1B0C1D0F108
:100C3000B1C1D1F1B2C1D2F1B3C1D3F1B4C1D4F1D8
:100C4000B5C1D5F1B6C1D6F1B7C1D7F1B8C1D8F1A8
:100C5000B9C1D9F1B7C5B9F5B8C5BAF5B9C5BBF5CC
:100C6000BAC5BCF5010155515B2756515C23E86AB2
:100C70005D230E2E44EF06F05CC157F15DC158F1C3
:100C80005B6B5C6B5D6B078E0201002F47EF0BF017
:100C90003C0E006F1D50E00BE00AE86612881BBE98
:100CA00002D01BB4108E00C10CF101C10DF102C1C4
:100CB0000EF103C10FF104C110F105C111F106C11C
:100CC00012F107C113F108C114F109C115F10AC1EC
:100CD00016F10BC117F134C135F181AAACEF06F062
:100CE00015A4F7EF06F005012F51000AD8B43AEF2A
:100CF00007F005012F51010AD8B4B6EF06F005013F
:100D00002F51020AD8B4F7EF06F005012F51030A5C
:100D1000D8B4F7EF06F005012F51040AD8B4F7EF65
:100D200006F005012F51050AD8B4F7EF06F00501CA
:100D30002F51060AD8B4F7EF06F005012F51070A24
:100D4000D8B4F7EF06F005012F51320AD8B4B4EF4A
:100D500006F02F6B3AEF07F000011650030AD8B4E3
:100D6000F7EF06F03AEF07F03AEF07F005015767A3
:100D7000C1EF06F05867C1EF06F05967C1EF06F002
:100D80005A67C5EF06F03AEF07F05BC500F15CC5A6
:100D900001F15DC502F15EC503F10101010E046FB1
:100DA000000E056F000E066F000E076F65EC2FF04A
:100DB00000C15BF501C15CF502C15DF503C15EF5E3
:100DC00001010067EBEF06F00167EBEF06F0026749
:100DD000EBEF06F003673AEF07F057C55BF558C530
:100DE0005CF559C55DF55AC55EF524EF07F00FBEF9
:100DF0000CEF07F010A011EF07F00101476708EFB3
:100E000007F0486708EF07F0496708EF07F04A67FF
:100E10000CEF07F011EF07F007AE11EF07F024EF2A
:100E200007F00501312F3AEF07F03C0E316F302FFC
:100E30003AEF07F00101000E626FE00E636FA50E3E
:100E4000646F010E656F138800011650000AD8B454
:100E500032EF07F000011650030AD8B437EF07F05D
:100E60003AEF07F00001010E166E3AEF07F00001AD
:100E7000040E166E0501666B37B740EF07F066810A
:100E80000CC100F10DC101F10EC102F10FC103F15E
:100E900010C104F111C105F112C106F113C107F12E
:100EA00014C108F115C109F116C10AF117C10BF1FE
:100EB00035C134F100C10CF101C10DF102C10EF1D7
:100EC00003C10FF104C110F105C111F106C112F106
:100ED00007C113F108C114F109C115F10AC116F1D6
:100EE0000BC117F134C135F101018E677FEF07F0B7
:100EF0008F677FEF07F090677FEF07F0916783EFD1
:100F000007F0B4EF07F092C100F193C101F194C171
:100F100002F195C103F10101010E046F000E056F8E
:100F2000000E066F000E076F65EC2FF000C192F106
:100F300001C193F102C194F103C195F10101006770
:100F4000A9EF07F00167A9EF07F00267A9EF07F023
:100F50000367B4EF07F08EC192F18FC193F190C196
:100F600094F191C195F10F80D57ED5BE6ED0D6CFCC
:100F700047F1D7CF48F145C149F1E86AE8CF4AF1D6
:100F8000138A1CBE02D01CA0108C109047C100F127
:100F900048C101F149C102F14AC103F101010A0E40
:100FA000046F000E056F000E066F000E076F65ECF4
:100FB0002FF003AF1080010154A7EBEF07F00F9A59
:100FC0000F9C0F9E0101000E5E6F600E5F6F3D0E65
:100FD000606F080E616F010147BFFBEF07F04867C4
:100FE000FBEF07F04967FBEF07F04A67FBEF07F0FD
:100FF000F28820EF08F0F2985E6B5F6B606B616BBC
:101000009A6B9B6B9C6B9D6B9E6B9F6BA06BA16B9C
:10101000A26BA36BA46BA56BA66BA76BA86BA96B4C
:10102000AA6BAB6BAC6BAD6BAE6BAF6BB06BB16BFC
:10103000B26BB36BB46BB56BB66BB76BB86BB96BAC
:10104000D76AD66A0101456B466B0CC100F10DC130
:1010500001F10EC102F10FC103F110C104F111C180
:1010600005F112C106F113C107F114C108F115C150
:1010700009F116C10AF117C10BF135C134F147EF7F
:101080000BF047EF0BF00201002FABEF0AF0D59EFB
:10109000D6CF47F1D7CF48F145C149F1E86AE8CF4B
:1010A0004AF1138AD76AD66A0101456B466BD58E21
:1010B0001D50E00BE00AE86612881BBE02D01BB48C
:1010C000108E1AAE1F8C00C10CF101C10DF102C1CE
:1010D0000EF103C10FF104C110F105C111F106C1F8
:1010E00012F107C113F108C114F109C115F10AC1C8
:1010F00016F10BC117F134C135F10FA0109A11B8D8
:101100008DEF08F00101620E046F010E056F000EF5
:10111000066F000E076F96EF08F00101A70E046F2F
:10112000020E056F000E066F000E076F47C100F13B
:1011300048C101F149C102F14AC103F165EC2FF048
:1011400003BFA9EF08F01CBE02D01CA0108C11B088
:101150000F800CC100F10DC101F10EC102F10FC1F0
:1011600003F110C104F111C105F112C106F113C15F
:1011700007F114C108F115C109F116C10AF117C12F
:101180000BF135C134F102013C0E006F00C10CF1CE
:1011900001C10DF102C10EF103C10FF104C110F143
:1011A00005C111F106C112F107C113F108C114F113
:1011B00009C115F10AC116F10BC117F134C135F19E
:1011C00081BAE6EF08F015B225EF09F015A025EF7A
:1011D00009F015A470EF09F005012F51000AD8B4E9
:1011E000B3EF09F005012F51010AD8B42FEF09F030
:1011F00005012F51020AD8B470EF09F005012F51F3
:10120000030AD8B470EF09F005012F51040AD8B4CD
:1012100070EF09F005012F51050AD8B470EF09F0FD
:1012200005012F51060AD8B470EF09F005012F51BE
:10123000070AD8B470EF09F005012F51320AD8B46B
:101240002DEF09F02F6BB3EF09F000011650030AE0
:10125000D8B470EF09F0B3EF09F0B3EF09F005016E
:1012600057673AEF09F058673AEF09F059673AEFD4
:1012700009F05A673EEF09F0B3EF09F05BC500F1E2
:101280005CC501F15DC502F15EC503F10101010E0E
:10129000046F000E056F000E066F000E076F65EC01
:1012A0002FF000C15BF501C15CF502C15DF503C122
:1012B0005EF50101006764EF09F0016764EF09F072
:1012C000026764EF09F00367B3EF09F057C55BF5F8
:1012D00058C55CF559C55DF55AC55EF59DEF09F039
:1012E0000FBE85EF09F010A08AEF09F001014767F2
:1012F00081EF09F0486781EF09F0496781EF09F054
:101300004A6785EF09F08AEF09F007AE8AEF09F026
:101310009DEF09F00501312FB3EF09F03C0E316F5D
:10132000302FB3EF09F00101000E626FE00E636F22
:10133000A50E646F010E656F138800011650000A38
:10134000D8B4ABEF09F000011650030AD8B4B0EFDF
:1013500009F0B3EF09F00001010E166EB3EF09F0CA
:101360000001040E166E0501666B37B7B9EF09F080
:1013700066810CC100F10DC101F10EC102F10FC176
:1013800003F110C104F111C105F112C106F113C13D
:1013900007F114C108F115C109F116C10AF117C10D
:1013A0000BF135C134F100C10CF101C10DF102C1E5
:1013B0000EF103C10FF104C110F105C111F106C115
:1013C00012F107C113F108C114F109C115F10AC1E5
:1013D00016F10BC117F134C135F101018E67F8EF39
:1013E00009F08F67F8EF09F09067F8EF09F091675F
:1013F000FCEF09F02DEF0AF092C100F193C101F169
:1014000094C102F195C103F10101010E046F000EB8
:10141000056F000E066F000E076F65EC2FF000C120
:1014200092F101C193F102C194F103C195F101015F
:10143000006722EF0AF0016722EF0AF0026722EF4D
:101440000AF003672DEF0AF08EC192F18FC193F17C
:1014500090C194F191C195F10F80109047C100F1B6
:1014600048C101F149C102F14AC103F101010A0E6B
:10147000046F000E056F000E066F000E076F65EC1F
:101480002FF003AF1080010154A753EF0AF00F9A19
:101490000F9C0F9E0101000E5E6F600E5F6F3D0E90
:1014A000606F080E616F47C100F148C101F149C189
:1014B00002F14AC103F10101140E046F050E056F1C
:1014C000000E066F000E076F65EC2FF003AF6CEF98
:1014D0000AF0F28891EF0AF0F2985E6B5F6B606B36
:1014E000616B9A6B9B6B9C6B9D6B9E6B9F6BA06BF8
:1014F000A16BA26BA36BA46BA56BA66BA76BA86B70
:10150000A96BAA6BAB6BAC6BAD6BAE6BAF6BB06B1F
:10151000B16BB26BB36BB46BB56BB66BB76BB86BCF
:10152000B96B0CC100F10DC101F10EC102F10FC187
:1015300003F110C104F111C105F112C106F113C18B
:1015400007F114C108F115C109F116C10AF117C15B
:101550000BF135C134F104008BB4B6EF0AF010ACD6
:10156000B6EF0AF08B84109CB7EF0AF08B94077CDF
:1015700007ACD2EF0AF0C274C2B4CCEF0AF0C3CF0A
:10158000B7F5C4CFB8F50501D890B833B733D890C4
:10159000B833B733D3EF0AF0C3CF55F1C4CF56F108
:1015A000D3EF0AF0C28207B445EF0BF047C14BF10D
:1015B00048C14CF149C14DF14AC14EF15EC162F1E1
:1015C0005FC163F160C164F161C165F113A8EBEF24
:1015D0000AF0138C13989AC1BAF19BC1BBF19CC15C
:1015E000BCF19DC1BDF19EC1BEF19FC1BFF1A0C1C3
:1015F000C0F1A1C1C1F1A2C1C2F1A3C1C3F1A4C193
:10160000C4F1A5C1C5F1A6C1C6F1A7C1C7F1A8C162
:10161000C8F1A9C1C9F1AAC1CAF1ABC1CBF1ACC132
:10162000CCF1ADC1CDF1AEC1CEF1AFC1CFF1B0C102
:10163000D0F1B1C1D1F1B2C1D2F1B3C1D3F1B4C1D2
:10164000D4F1B5C1D5F1B6C1D6F1B7C1D7F1B8C1A2
:10165000D8F1B9C1D9F1B7C5B9F5B8C5BAF5B9C5A9
:10166000BBF5BAC5BCF5010155515B2756515C234A
:10167000E86A5D230E2E45EF0BF05CC157F15DC1AA
:1016800058F15B6B5C6B5D6B078E47EF0BF002C034
:10169000E0FF005001C0D8FF1000A6B24DEF0BF0E4
:1016A0000CC0A9FF0BC0A8FFA69EA69CA684F29E14
:1016B000550EA76EAA0EA76EA682F28EA694A6B2AB
:1016C0005FEF0BF00C2A1200A96EA69EA69CA680C6
:1016D000A8500C2A120004012C0E826F93EC0EF01D
:1016E00060EC30F00C5064EC0BF0E8CF00F10C50E3
:1016F00064EC0BF0E8CF01F101AF84EF0BF00101D6
:10170000FF0E026FFF0E036F03EC30F0296790EFBE
:101710000BF00401200E826F93EC0EF095EF0BF0AE
:1017200004012D0E826F93EC0EF00DEC2EF01200E2
:101730001594076A0F6A106A116A126A136A166AA8
:101740000F010D0EC16E860EC06E030EC26E0F012C
:10175000680E896E130E926E080E8A6EF30E936EEB
:101760008B6A900E946EC80E64EC0BF0E8CFE8FF25
:101770001098E8A0108810A805D00E0E256E8E0EC9
:10178000266E04D00F0E256E8F0E266EF8EC30F00C
:10179000F18EF19EFC0E64EC0BF0E8CF0BF00BA089
:1017A00011800BA211820BA411840BA81188C90E01
:1017B00064EC0BF0E8CF1AF0CA0E64EC0BF0E8CF43
:1017C0001BF0CB0E64EC0BF0E8CF1CF0CC0E64ECFD
:1017D0000BF0E8CF1DF0FB0E64EC0BF0E8CF37F018
:1017E000CE0E64EC0BF0E8CF14F0CD0E64EC0BF0F1
:1017F000E8CF36F01F6A206A0E6A01015B6B5C6BF2
:101800005D6B576B586BF29A0101476B486B496BE4
:101810004A6B4B6B4C6B4D6B4E6B4F6B506B516B04
:10182000526B456B466BD76AD66A0F01280ED56E90
:10183000F28A9D90B00ECD6E01015E6B5F6B606BA6
:10184000616B626B636B646B656B666B676B686B1C
:10185000696B536B546BCF6ACE6A0F9A0F9C0F9EC5
:101860009D80760ECA6E9D8202013C0E006FCC6A8E
:10187000160E64EC0BF0E8CF00F1170E64EC0BF0E1
:10188000E8CF01F1180E64EC0BF0E8CF02F1190E6D
:1018900064EC0BF0E8CF03F1010103AF6AEF0CF049
:1018A00060EC30F0160E0C6E00C10BF04DEC0BF03E
:1018B000170E0C6E01C10BF04DEC0BF0180E0C6EF8
:1018C00002C10BF04DEC0BF0190E0C6E03C10BF0C6
:1018D0004DEC0BF000C18EF101C18FF102C190F10E
:1018E00003C191F100C192F101C193F102C194F1E0
:1018F00003C195F11A0E64EC0BF0E8CF00F11B0E5A
:1019000064EC0BF0E8CF01F11C0E64EC0BF0E8CFB7
:1019100002F11D0E64EC0BF0E8CF03F1010103AFFF
:10192000C0EF0CF060EC30F01A0E0C6E00C10BF042
:101930004DEC0BF01B0E0C6E01C10BF04DEC0BF0DF
:101940001C0E0C6E02C10BF04DEC0BF01D0E0C6E5C
:1019500003C10BF04DEC0BF01A0E64EC0BF0E8CF6A
:1019600000F11B0E64EC0BF0E8CF01F11C0E64ECEF
:101970000BF0E8CF02F11D0E64EC0BF0E8CF03F1A1
:1019800000C196F101C197F102C198F103C199F12B
:10199000240EAC6E900EAB6E240EAC6E080EB86EBC
:1019A000000EB06E1F0EAF6E0401806B816B0F01D5
:1019B000900EAB6E0F019D8A0301806B816BC26B31
:1019C0008B929DEC35F09DEC35F057EC37F07BECCD
:1019D00033F0200E64EC0BF0E8CF2FF505012F510A
:1019E000FF0AD8A4FBEF0CF02F6B200E0C6E2FC556
:1019F0000BF04DEC0BF00501010E306F3C0E316F1A
:101A0000250E64EC0BF0E8CF00F1260E64EC0BF031
:101A1000E8CF01F1270E64EC0BF0E8CF02F1280EBD
:101A200064EC0BF0E8CF03F1010103AF32EF0DF0EE
:101A300060EC30F0250E0C6E00C10BF04DEC0BF09D
:101A4000260E0C6E01C10BF04DEC0BF0270E0C6E48
:101A500002C10BF04DEC0BF0280E0C6E03C10BF025
:101A60004DEC0BF000C157F501C158F502C159F515
:101A700003C15AF500C15BF501C15CF502C15DF51A
:101A800003C15EF5290E64EC0BF0E8CF5FF50501AC
:101A900060515F5DD8A05FC560F5210E64EC0BF06E
:101AA000E8CF00F1220E64EC0BF0E8CF01F1230E39
:101AB00064EC0BF0E8CF02F1240E64EC0BF0E8CFFD
:101AC00003F1010103AF93EF0DF060EC30F0210E54
:101AD0000C6E00C10BF04DEC0BF0220E0C6E01C130
:101AE0000BF04DEC0BF0230E0C6E02C10BF04DEC25
:101AF0000BF0240E0C6E03C10BF04DEC0BF0210E1D
:101B000064EC0BF0E8CF00F1220E64EC0BF0E8CFB0
:101B100001F1230E64EC0BF0E8CF02F1240E64EC2B
:101B20000BF0E8CF03F100C161F501C162F502C11C
:101B300063F503C164F5C3EC32F0A9EC31F001ECBC
:101B400031F01590C70E64EC0BF0E8CF00F1010105
:101B500000B1AEEF0DF01592AFEF0DF0158281AA36
:101B6000BDEF0DF015B4B8EF0DF01580BDEF0DF021
:101B700096EC37F015A0F9EF37F007900001F28EE0
:101B8000F28C12AE03D012BC6AEF19F007B09AEFD4
:101B90002CF00FB096EF25F010BE96EF25F012B89E
:101BA00096EF25F000011650010AD8B49DEF1DF004
:101BB00081BAE3EF0DF000011650040AD8B416EF15
:101BC0001CF0E9EF0DF000011650040AD8B4D2EF72
:101BD0001DF00301805181197F0BD8B49AEF2CF0CE
:101BE00013EE00F081517F0BE126812BE7CFE8FF58
:101BF000E00BD8B49AEF2CF023EE82F0C2513F0BE9
:101C0000D926E7CFDFFFC22BDF50780AD8A49AEF9E
:101C10002CF0078092C100F193C101F194C102F14F
:101C200095C103F10101040E046F000E056F000E53
:101C3000066F000E076F65EC2FF000AF29EF0EF076
:101C40000101030E926F000E936F000E946F000E51
:101C5000956F03018251720AD8B417EF25F08251B3
:101C6000520AD8B417EF25F08251750AD8B417EF8D
:101C700025F08251680AD8B4A7EF0EF08251630AAA
:101C8000D8B454EF29F08251690AD8B4D5EF20F0C6
:101C900082517A0AD8B4E8EF21F08251490AD8B4C7
:101CA00074EF20F08251500AD8B492EF1FF08251A5
:101CB000700AD8B4D5EF1FF08251540AD8B400EF9F
:101CC00020F08251740AD8B446EF20F08251410AC4
:101CD000D8B4ACEF0FF082514B0AD8B4A9EF0EF094
:101CE00082516D0AD8B41CEF14F082514D0AD8B459
:101CF00035EF14F08251730AD8B447EF24F08251C3
:101D0000530AD8B4ACEF24F082514C0AD8B4C4EFD3
:101D100014F08251590AD8B46DEF13F012AE01D00D
:101D2000128C8BEF29F0040114EE00F080517F0B30
:101D3000E12682C4E7FF802B120004010D0E826FA2
:101D400093EC0EF00A0E826F93EC0EF0120089EF06
:101D500029F004014B0E826F93EC0EF004012C0E5F
:101D6000826F93EC0EF081B802D036B630D003010A
:101D70008351430AD8B4EEEF0EF003018351630A96
:101D8000D8B4F0EF0EF003018351520AD8B4F2EF49
:101D90000EF003018351720AD8B4F4EF0EF0030180
:101DA0008351470AD8B4F6EF0EF003018351670A56
:101DB000D8B4F8EF0EF003018351540AD8B4FAEF07
:101DC0000EF003018351740AD8B46AEF0FF00301D7
:101DD0008351550AD8B4FCEF0EF083D036807BD007
:101DE000369079D0368277D0369275D0368473D0DB
:101DF000369471D036866FD084C330F185C331F10B
:101E000086C332F187C333F10101296BAEEC30F0A8
:101E100025EC30F000C104F101C105F102C106F169
:101E200003C107F1A1EC30F0200EF86EF76AF66AF4
:101E30000900F5CF2CF10900F5CF2DF10900F5CF00
:101E40002EF10900F5CF2FF10900F5CF30F109008F
:101E5000F5CF31F10900F5CF32F10900F5CF33F1BB
:101E60000101296BAEEC30F025EC30F065EC2FF081
:101E70000101006743EF0FF0016743EF0FF00267C6
:101E800043EF0FF0036701D025D004014E0E826F9F
:101E900093EC0EF004016F0E826F93EC0EF00401D0
:101EA0004D0E826F93EC0EF00401610E826F93EC85
:101EB0000EF00401740E826F93EC0EF00401630EB9
:101EC000826F93EC0EF00401680E826F93EC0EF0BB
:101ED00089EF29F03696CD0E0C6E36C00BF04DEC26
:101EE0000BF0CD0E64EC0BF0E8CF36F036B006D038
:101EF0000401630E826F93EC0EF005D00401430ED3
:101F0000826F93EC0EF036B206D00401720E826F2F
:101F100093EC0EF005D00401520E826F93EC0EF09C
:101F200036B406D00401670E826F93EC0EF005D034
:101F30000401470E826F93EC0EF036B606D0040112
:101F4000740E826F93EC0EF005D00401540E826F74
:101F500093EC0EF089EF29F00401410E826F93ECAF
:101F60000EF003018351310AD8B48DEF12F0030152
:101F70008351320AD8B4BDEF11F003018351330A03
:101F8000D8B446EF11F003018351340AD8B436EFC8
:101F900010F003018351350AD8B4D6EF0FF00401D5
:101FA0003F0E826F93EC0EF089EF29F0030184510C
:101FB000300AD8B4FCEF0FF003018451310AD8B4D1
:101FC000FFEF0FF003018451650AD8B4F0EF0FF072
:101FD00003018451640AD8B4F3EF0FF000EF10F05E
:101FE0003790F4EF0FF03780FB0E0C6E37C00BF01C
:101FF0004DEC0BF000EF10F08B9000EF10F08B80A9
:102000000401350E826F93EC0EF004012C0E826FEA
:1020100093EC0EF08BB014EF10F00401300E826FD1
:1020200093EC0EF019EF10F00401310E826F93EC77
:102030000EF004012C0E826F93EC0EF0FB0E64EC9C
:102040000BF0E8CF37F037A02DEF10F00401640E4D
:10205000826F93EC0EF032EF10F00401650E826F88
:1020600093EC0EF034EF10F089EF29F0CC0E64EC15
:102070000BF0E8CF0BF004012C0E826F93EC0EF006
:1020800003018451310AD8B45AEF10F0030184518E
:10209000300AD8B45CEF10F0030184514D0AD8B473
:1020A00066EF10F003018451540AD8B46DEF10F0BC
:1020B00084EF10F08A8401D08A940BAE04D00BAC6C
:1020C00002D00BBA21D0E00E0B1218D01F0E0B1647
:1020D0008539E844E00B0B1211D0E00E0B16A1EC91
:1020E00030F085C332F186C333F10101296BAEECC8
:1020F00030F025EC30F000511F0B0B12CC0E0C6EA3
:102100000BC00BF04DEC0BF00401340E826F93EC1E
:102110000EF004012C0E826F93EC0EF0CC0E64ECEA
:102120000BF0E8CF1DF08AB406D00401300E826FA8
:1021300093EC0EF005D00401310E826F93EC0EF09B
:1021400004012C0E826F93EC0EF01D38E840070B53
:10215000E8CF82F40401300E822793EC0EF00401E4
:102160002C0E826F93EC0EF060EC30F01D501F0BC4
:10217000E8CF00F103EC30F032C182F40401300EFC
:10218000822793EC0EF033C182F40401300E8227D3
:1021900093EC0EF004012C0E826F93EC0EF060ECC9
:1021A00030F030C000F100AF0BD0FF0E016FFF0E1A
:1021B000026FFF0E036F04012D0E826F93EC0EF081
:1021C00003EC30F031C182F40401300E822793EC2D
:1021D0000EF032C182F40401300E822793EC0EF02F
:1021E00033C182F40401300E822793EC0EF0040117
:1021F0002C0E826F93EC0EF060EC30F02FC000F1EB
:1022000003EC30F031C182F40401300E822793ECEC
:102210000EF032C182F40401300E822793EC0EF0EE
:1022200033C182F40401300E822793EC0EF00401D6
:102230002C0E826F93EC0EF060EC30F031C000F1A8
:1022400000AF0BD0FF0E016FFF0E026FFF0E036F8A
:1022500004012D0E826F93EC0EF003EC30F031C1CF
:1022600082F40401300E822793EC0EF032C182F426
:102270000401300E822793EC0EF033C182F4040186
:10228000300E822793EC0EF089EF29F0CB0E64EC30
:102290000BF0E8CF0BF004012C0E826F93EC0EF0E4
:1022A00003018451450AD8B46AEF11F00301845147
:1022B000440AD8B46DEF11F003018451300AD8B448
:1022C00070EF11F003018451310AD8B474EF11F0AA
:1022D0007FEF11F00B9E79EF11F00B8E79EF11F07B
:1022E000FC0E0B1679EF11F0FC0E0B160B8079EF3C
:1022F00011F0CB0E0C6E0BC00BF04DEC0BF004018B
:10230000330E826F93EC0EF004012C0E826F93EC6F
:102310000EF0CB0E64EC0BF0E8CF1CF01CBE98EF77
:1023200011F00401450E826F93EC0EF09DEF11F059
:102330000401440E826F93EC0EF004012C0E826FA8
:1023400093EC0EF00401300E826F93EC0EF004015A
:102350002C0E826F93EC0EF01CB0B6EF11F004015E
:10236000300E826F93EC0EF0BBEF11F00401310ED2
:10237000826F93EC0EF089EF29F0CA0E64EC0BF03B
:10238000E8CF0BF004012C0E826F93EC0EF00301EA
:102390008451450AD8B4F9EF11F003018451440A7D
:1023A000D8B4FCEF11F0030184514D0AD8B405EF05
:1023B00012F003018451410AD8B4FFEF11F0030178
:1023C0008451460AD8B402EF12F003018451560A30
:1023D000D8B40DEF12F003018451500AD8B418EFAD
:1023E00012F003018451520AD8B41BEF12F024EF0B
:1023F00012F00B9E1EEF12F00B8E1EEF12F00B9CD4
:102400001EEF12F00B8C1EEF12F0FC0E0B1685C3A4
:10241000E8FF030B0B121EEF12F0C70E0B1685C35D
:10242000E8FF070BE846E846E8460B121EEF12F0FD
:102430000B841EEF12F00B941EEF12F0CA0E0C6EFE
:102440000BC00BF04DEC0BF0CA0E64EC0BF0E8CFB8
:102450001BF00401320E826F93EC0EF004012C0E7F
:10246000826F93EC0EF01BBE3DEF12F00401450E9F
:10247000826F93EC0EF042EF12F00401440E826F73
:1024800093EC0EF004012C0E826F93EC0EF01BC047
:10249000E8FF030BE8CF82F40401300E822793ECAF
:1024A0000EF004012C0E826F93EC0EF01BBC60EF5B
:1024B00012F00401410E826F93EC0EF065EF12F002
:1024C0000401460E826F93EC0EF004012C0E826F15
:1024D00093EC0EF01BC0E8FF380BE842E842E842FC
:1024E000E8CF82F40401300E822793EC0EF0040151
:1024F0002C0E826F93EC0EF01BB486EF12F00401E9
:10250000520E826F93EC0EF08BEF12F00401500E1E
:10251000826F93EC0EF089EF29F0C90E64EC0BF09A
:10252000E8CF0BF004012C0E826F93EC0EF0030148
:102530008451450AD8B4ABEF12F003018451440A28
:10254000D8B4AEEF12F0030184514D0AD8B4B1EF04
:1025500012F0BFEF12F00B9EB9EF12F00B8EB9EF35
:1025600012F0F80E0B1685C3E8FF070B0B12B9EF3C
:1025700012F0C90E0C6E0BC00BF04DEC0BF0040109
:10258000310E826F93EC0EF004012C0E826F93ECEF
:102590000EF0C90E64EC0BF0E8CF1AF01ABE06D0AC
:1025A0000401450E826F93EC0EF005D00401440E39
:1025B000826F93EC0EF004012C0E826F93EC0EF000
:1025C0001AC0E8FF070BE8CF82F40401300E82271F
:1025D00093EC0EF004012C0E826F93EC0EF007804A
:1025E00060EC30F02BC0E8FF003B00430043030BDE
:1025F00003EC30F033C182F40401300E822793ECF7
:102600000EF004012C0E826F93EC0EF060EC30F0B3
:102610002BC001F1019F019D2CC000F1010103ECD1
:1026200030F02FC182F40401300E822793EC0EF0BB
:1026300030C182F40401300E822793EC0EF031C1D8
:1026400082F40401300E822793EC0EF032C182F442
:102650000401300E822793EC0EF033C182F40401A2
:10266000300E822793EC0EF004012C0E826F93EC57
:102670000EF060EC30F02DC001F12EC000F1D890CA
:1026800001330033D89001330033010103EC30F003
:102690002FC182F40401300E822793EC0EF030C17A
:1026A00082F40401300E822793EC0EF031C182F4E3
:1026B0000401300E822793EC0EF032C182F4040143
:1026C000300E822793EC0EF033C182F40401300EF9
:1026D000822793EC0EF089EF29F0FC0E64EC0BF0EE
:1026E000E8CF0BF003018351520AD8B4A4EF13F0E2
:1026F00003018351720AD8B4A7EF13F00301835189
:10270000500AD8B4AAEF13F003018351700AD8B469
:10271000ADEF13F003018351550AD8B4B0EF13F0B5
:1027200003018351750AD8B4B3EF13F00301835149
:10273000430AD8B4BCEF13F003018351630AD8B441
:10274000BFEF13F0C8EF13F00B90C2EF13F00B8044
:10275000C2EF13F00B92C2EF13F00B82C2EF13F033
:102760000B94C2EF13F00B84C2EF13F00B96C2EF81
:1027700013F00B86C2EF13F00B98C2EF13F00B8827
:10278000C2EF13F0FC0E0C6E0BC00BF04DEC0BF017
:102790000401590E826F93EC0EF011901192119476
:1027A0001198FC0E64EC0BF0E8CF0BF00BA011803D
:1027B0000BA211820BA411840BA8118811A0E8EFC1
:1027C00013F00401520E826F93EC0EF0EDEF13F054
:1027D0000401720E826F93EC0EF011A8F7EF13F064
:1027E0000401430E826F93EC0EF0FCEF13F0040132
:1027F000630E826F93EC0EF011A206EF14F0040149
:10280000500E826F93EC0EF00BEF14F00401700E7B
:10281000826F93EC0EF011A415EF14F00401550E25
:10282000826F93EC0EF01AEF14F00401750E826FB4
:1028300093EC0EF089EF29F004016D0E826F93EC9A
:102840000EF003018351300AD8B474EF14F0030181
:102850008351310AD8B487EF14F003018351320A4F
:10286000D8B49AEF14F08BEF29F004014D0E826F6B
:1028700093EC0EF0A1EC30F084C331F185C332F15A
:1028800086C333F10101296BAEEC30F025EC30F05A
:1028900003018351300AD8B45CEF14F00301835173
:1028A000310AD8B464EF14F003018351320AD8B46A
:1028B0006CEF14F08BEF29F0FD0E0C6E00C10BF0E5
:1028C0004DEC0BF074EF14F0FE0E0C6E00C10BF02B
:1028D0004DEC0BF087EF14F0FF0E0C6E00C10BF007
:1028E0004DEC0BF09AEF14F00401300E826F93EC74
:1028F0000EF004012C0E826F93EC0EF060EC30F0C1
:10290000FD0E64EC0BF0E8CF00F1ABEF14F0040126
:10291000310E826F93EC0EF004012C0E826F93EC5B
:102920000EF060EC30F0FE0E64EC0BF0E8CF00F13E
:10293000ABEF14F00401320E826F93EC0EF060ECFA
:1029400030F004012C0E826F93EC0EF0FF0E64EC5D
:102950000BF0E8CF00F103EC30F031C182F4040158
:10296000300E822793EC0EF032C182F40401300E57
:10297000822793EC0EF033C182F40401300E8227DB
:1029800093EC0EF089EF29F003018351300AD8B49B
:1029900017EF1AF003018351310AD8B444EF1BF04A
:1029A00003018351320AD8B4B2EF1BF00301835103
:1029B000330AD8B4C2EF1BF003018351340AD8B4F0
:1029C0001DEF1CF003018351350AD8B4E3EF1DF06D
:1029D00003018351360AD8B411EF1EF0030183516D
:1029E000370AD8B4EFEF17F003018351380AD8B48F
:1029F0008DEF18F003018351440AD8B41CEF16F090
:102A000003018351640AD8B43BEF16F003018351EC
:102A1000460AD8B4F6EF1CF0030183514D0AD8B42E
:102A200068EF16F0030183516D0AD8B482EF16F0F7
:102A3000030183515A0AD8B4BEEF1AF0030183513F
:102A4000490AD8B411EF1FF003018351500AD8B4DA
:102A500043EF1EF003018351540AD8B4BCEF1EF0BB
:102A600003018351630AD8B4A2EF16F00301835126
:102A7000430AD8B49AEF17F003018351730AD8B40C
:102A8000A0EF16F003018351610AD8B469EF15F085
:102A900003018351650AD8B467EF1AF0030183512B
:102AA000450AD8B475EF1AF003018351620AD8B40D
:102AB00083EF1AF003018351420AD8B491EF1AF060
:102AC00003018351760AD8B49FEF1AF0D8A48BEF94
:102AD00029F004014C0E826F93EC0EF00401610E9C
:102AE000826F93EC0EF0A9EC31F004012C0E826F92
:102AF00093EC0EF060EC30F0AFC500F1010103EC97
:102B000030F031C182F40401300E822793EC0EF0D4
:102B100032C182F40401300E822793EC0EF033C1EF
:102B200082F40401300E822793EC0EF004012C0E87
:102B3000826F93EC0EF060EC30F0B0C500F1010153
:102B400003EC30F031C182F40401300E822793ECA3
:102B50000EF032C182F40401300E822793EC0EF0A5
:102B600033C182F40401300E822793EC0EF004018D
:102B70002C0E826F93EC0EF060EC30F0B1C500F1DA
:102B8000010103EC30F031C182F40401300E8227E0
:102B900093EC0EF032C182F40401300E822793ECE4
:102BA0000EF033C182F40401300E822793EC0EF054
:102BB00004012C0E826F93EC0EF060EC30F0B2C585
:102BC00000F1010103EC30F031C182F40401300E58
:102BD000822793EC0EF032C182F40401300E82277A
:102BE00093EC0EF033C182F40401300E822793EC93
:102BF0000EF004012C0E826F93EC0EF060EC30F0BE
:102C0000B6C500F1010103EC30F031C182F40401DA
:102C1000300E822793EC0EF032C182F40401300EA4
:102C2000822793EC0EF033C182F40401300E822728
:102C300093EC0EF03FEF1EF003018451300AD8B43C
:102C400028EF16F003018451310AD8B42BEF16F0A7
:102C500015922CEF16F01582C70E64EC0BF0E8CF3E
:102C600000F10101008115A20091C70E0C6E00C198
:102C70000BF04DEC0BF0C70E64EC0BF0E8CF00F15D
:102C8000010100B147EF16F0159248EF16F01582DA
:102C900004014C0E826F93EC0EF00401640E826FFF
:102CA00093EC0EF004012C0E826F93EC0EF015B233
:102CB00061EF16F00401300E826F93EC0EF066EFB8
:102CC00016F00401310E826F93EC0EF089EF29F0BB
:102CD000A1EC30F084C333F1AEEC30F025EC30F0F1
:102CE000200E0C6E00C10BF04DEC0BF000C12FF567
:102CF00005012F51000A06E005012F51010A02E0EB
:102D000043EC32F004014C0E826F93EC0EF00401A0
:102D10004D0E826F93EC0EF004012C0E826F93EC3B
:102D20000EF060EC30F02FC500F103EC30F033C151
:102D300082F40401300E822793EC0EF03FEF1EF078
:102D4000F9EF37F004014C0E826F93EC0EF00401A2
:102D5000630E826F93EC0EF001EC31F004012C0E47
:102D6000826F93EC0EF0B7EC16F03FEF1EF060ECC4
:102D700030F0B5C500F10101003B0F0E001703EC68
:102D800030F033C182F40401300E822793EC0EF050
:102D9000B5C500F101010F0E0101001703EC30F081
:102DA00033C182F40401300E822793EC0EF004014B
:102DB0002D0E826F93EC0EF0B4C500F10101003BC3
:102DC0000F0E001703EC30F033C182F40401300E13
:102DD000822793EC0EF0B4C500F101010F0E010142
:102DE000001703EC30F033C182F40401300E822767
:102DF00093EC0EF004012D0E826F93EC0EF0B3C530
:102E000000F10101003B0F0E001703EC30F033C15D
:102E100082F40401300E822793EC0EF0B3C500F16A
:102E200001010F0E0101001703EC30F033C182F4F1
:102E30000401300E822793EC0EF00401200E826F05
:102E400093EC0EF0B2C500F10F0E0101001703EC78
:102E500030F033C182F40401300E822793EC0EF07F
:102E60000401200E826F93EC0EF0B1C500F1010158
:102E70000101003B0F0E001703EC30F033C182F468
:102E80000401300E822793EC0EF0B1C500F1010170
:102E90000F0E0101001703EC30F033C182F404017E
:102EA000300E822793EC0EF004013A0E826F93EC01
:102EB0000EF0B0C500F10101003B0F0E001703EC4E
:102EC00030F033C182F40401300E822793EC0EF00F
:102ED000B0C500F101010F0E0101001703EC30F045
:102EE00033C182F40401300E822793EC0EF004010A
:102EF0003A0E826F93EC0EF0AFC500F10101003B7A
:102F00000F0E001703EC30F033C182F40401300ED1
:102F1000822793EC0EF0AFC500F101010F0E0017F0
:102F200003EC30F033C182F40401300E822793ECBD
:102F30000EF0120084C3E8FF0F0BE83AE8CFB5F5B6
:102F400085C3E8FF0F0B0501B51387C3E8FF0F0B1F
:102F5000E83AE8CFB4F588C3E8FF0F0B0501B413D6
:102F60008AC3E8FF0F0BE83AE8CFB3F58BC3E8FF5D
:102F70000F0B0501B3138DC3E8FF0F0BE8CFB2F5BC
:102F80008FC3E8FF0F0BE83AE8CFB1F590C3E8FF35
:102F90000F0B0501B11392C3E8FF0F0BE83AE8CF1E
:102FA000B0F593C3E8FF0F0B0501B01395C3E8FF1D
:102FB0000F0BE83AE8CFAFF596C3E8FF0F0B05011A
:102FC000AF135CEC31F004014C0E826F93EC0EF009
:102FD0000401430E826F93EC0EF0ACEF16F0078401
:102FE00004014C0E826F93EC0EF00401370E826FD9
:102FF00093EC0EF004012C0E826F93EC0EF00501A1
:103000002E51130A06E005012E51170A0DE08AEF32
:1030100018F00101000E006F000E016F100E026F1C
:10302000000E036F1DEF18F00101000E006F000E7F
:10303000016F000E026F010E036F03EC30F02AC126
:1030400082F40401300E822793EC0EF02BC182F43F
:103050000401300E822793EC0EF02CC182F404019F
:10306000300E822793EC0EF02DC182F40401300E55
:10307000822793EC0EF02EC182F40401300E8227D9
:1030800093EC0EF02FC182F40401300E822793ECF2
:103090000EF030C182F40401300E822793EC0EF062
:1030A00031C182F40401300E822793EC0EF032C15C
:1030B00082F40401300E822793EC0EF033C182F4C7
:1030C0000401300E822793EC0EF004012C0E826F67
:1030D00093EC0EF00101100E006F000E016F000E58
:1030E000026F000E036F03EC30F031C182F4040173
:1030F000300E822793EC0EF032C182F40401300EC0
:10310000822793EC0EF033C182F40401300E822743
:1031100093EC0EF007943FEF1EF00501216B226B3C
:10312000236B246B04014C0E826F93EC0EF00401B0
:10313000380E826F93EC0EF004012C0E826F93EC2C
:103140000EF00101100E006F000E016F000E026FF5
:10315000000E036F03EC30F02AC182F40401300E3C
:10316000822793EC0EF02BC182F40401300E8227EB
:1031700093EC0EF02CC182F40401300E822793EC04
:103180000EF02DC182F40401300E822793EC0EF074
:103190002EC182F40401300E822793EC0EF02FC171
:1031A00082F40401300E822793EC0EF030C182F4D9
:1031B0000401300E822793EC0EF031C182F4040139
:1031C000300E822793EC0EF032C182F40401300EEF
:1031D000822793EC0EF033C182F40401300E822773
:1031E00093EC0EF004012C0E826F93EC0EF025C5CB
:1031F00000F126C501F127C502F128C503F101013F
:10320000100E046F000E056F000E066F000E076FA4
:1032100096EC2FF000C133F501C134F502C135F54C
:1032200003C136F503EC30F02AC182F40401300EFC
:10323000822793EC0EF02BC182F40401300E82271A
:1032400093EC0EF02CC182F40401300E822793EC33
:103250000EF02DC182F40401300E822793EC0EF0A3
:103260002EC182F40401300E822793EC0EF02FC1A0
:1032700082F40401300E822793EC0EF030C182F408
:103280000401300E822793EC0EF031C182F4040168
:10329000300E822793EC0EF032C182F40401300E1E
:1032A000822793EC0EF033C182F40401300E8227A2
:1032B00093EC0EF09DEC0EF00501336767EF19F00B
:1032C000346767EF19F0356767EF19F0366702D09A
:1032D00006EF1AF0129E129C21C500F122C501F1E1
:1032E00023C502F124C503F1899A400EC76E200E52
:1032F000C66E9E96C69E0B0EC96EFF0E9EB602D07F
:10330000E82EFCD79E96C69E02C1C9FFFF0E9EB650
:1033100002D0E82EFCD79E96C69E01C1C9FFFF0EC3
:103320009EB602D0E82EFCD79E96C69E00C1C9FF6D
:10333000FF0E9EB602D0E82EFCD79E96C69EC952BE
:10334000FF0E9EB602D0E82EFCD70501100E326F9C
:10335000040114EE00F080517F0BE1269E96C69E7C
:10336000C952FF0E9EB602D0E82EFCD7C9CFE7FFA8
:103370000401802B0501322FA8EF19F0898A33C58B
:1033800000F134C501F135C502F136C503F1010183
:10339000010E046F000E056F000E066F000E076F22
:1033A00065EC2FF000C133F501C134F502C135F5EC
:1033B00003C136F505013367E5EF19F03467E5EF32
:1033C00019F03567E5EF19F0366702D006EF1AF00D
:1033D00021C500F122C501F123C502F124C503F185
:1033E0000101100E046F000E056F000E066F000E37
:1033F000076F6AEC2FF000C121F501C122F502C16F
:1034000023F503C124F5128E8BEF29F00401450E3C
:10341000826F93EC0EF004014F0E826F93EC0EF06E
:103420000401460E826F93EC0EF03FEF1EF007840E
:1034300057EC37F060EC30F02DC500F103EC30F0C4
:1034400004014C0E826F93EC0EF00401300E826F7B
:1034500093EC0EF004012C0E826F93EC0EF031C150
:1034600082F40401300E822793EC0EF032C182F414
:103470000401300E822793EC0EF033C182F4040174
:10348000300E822793EC0EF004012C0E826F93EC29
:103490000EF060EC30F02EC500F103EC30F031C1DD
:1034A00082F40401300E822793EC0EF032C182F4D4
:1034B0000401300E822793EC0EF033C182F4040134
:1034C000300E822793EC0EF007943FEF1EF00401BC
:1034D0004C0E826F93EC0EF00401650E826F93EC3C
:1034E0000EF01FEC33F03FEF1EF004014C0E826F24
:1034F00093EC0EF00401450E826F93EC0EF036EC67
:1035000033F03FEF1EF004014C0E826F93EC0EF08F
:103510000401620E826F93EC0EF064EC33F03FEF27
:103520001EF004014C0E826F93EC0EF00401420E6B
:10353000826F93EC0EF04DEC33F03FEF1EF0040180
:103540004C0E826F93EC0EF00401760E826F93ECBA
:103550000EF004012C0E826F93EC0EF010A807D031
:103560000401310E826F93EC0EF03FEF1EF0040168
:10357000300E826F93EC0EF03FEF1EF004014C0E04
:10358000826F93EC0EF004015A0E826F93EC0EF0F2
:1035900004012C0E826F93EC0EF057EC37F060ECC8
:1035A00030F005012E51130A06E005012E51170ACD
:1035B0000DE0EFEF1AF00101000E006F000E016F39
:1035C000100E026F000E036FEFEF1AF00101000EF4
:1035D000006F000E016F000E026F010E036F0101FC
:1035E000100E046F000E056F000E066F000E076FC1
:1035F00096EC2FF003EC30F02AC182F40401300E77
:10360000822793EC0EF02BC182F40401300E822746
:1036100093EC0EF02CC182F40401300E822793EC5F
:103620000EF02DC182F40401300E822793EC0EF0CF
:103630002EC182F40401300E822793EC0EF02FC1CC
:1036400082F40401300E822793EC0EF030C182F434
:103650000401300E822793EC0EF031C182F4040194
:10366000300E822793EC0EF032C182F40401300E4A
:10367000822793EC0EF033C182F40401300E8227CE
:1036800093EC0EF03FEF1EF0078404014C0E826FA6
:1036900093EC0EF00401310E826F93EC0EF00401F6
:1036A0002C0E826F93EC0EF025C500F126C501F1BA
:1036B00027C502F128C503F10101100E046F000EA9
:1036C000056F000E066F000E076F96EC2FF003ECEF
:1036D00030F02AC182F40401300E822793EC0EF000
:1036E0002BC182F40401300E822793EC0EF02CC122
:1036F00082F40401300E822793EC0EF02DC182F487
:103700000401300E822793EC0EF02EC182F40401E6
:10371000300E822793EC0EF02FC182F40401300E9C
:10372000822793EC0EF030C182F40401300E822720
:1037300093EC0EF031C182F40401300E822793EC39
:103740000EF032C182F40401300E822793EC0EF0A9
:1037500033C182F40401300E822793EC0EF00794FB
:103760003FEF1EF0078404014C0E826F93EC0EF0C5
:103770000401320E826F93EC0EF053EC35F0079497
:103780003FEF1EF0078437B0C8EF1BF0DBEF1BF0F4
:10379000010E166E04014C0E826F93EC0EF00401C4
:1037A000330E826F93EC0EF0B0EC35F0000E166E17
:1037B00007944FEF1BF0020E166EB0EC35F08B80C5
:1037C0000501010E306F3C0E316F01015E6B5F6BC6
:1037D000606B616B626B636B646B656B666B676B75
:1037E000686B696B536B546BCF6ACE6A0F9A0F9CF0
:1037F0000F9E030E166E04014C0E826F93EC0EF0BA
:103800000401330E826F93EC0EF004012C0E826FD4
:1038100093EC0EF004012D0E826F93EC0EF0040178
:10382000310E826F93EC0EF089EF29F0B0EC35F099
:10383000000E166E8B908BEF29F0078404014C0E5E
:10384000826F93EC0EF00401340E826F93EC0EF055
:1038500004012C0E826F93EC0EF0A1EC30F084C3C7
:103860002AF185C32BF186C32CF187C32DF188C3C0
:103870002EF189C32FF18AC330F18BC331F18CC390
:1038800032F18DC333F10101296BAEEC30F025EC40
:1038900030F0100E046F000E056F000E066F000E64
:1038A000076F76EC2FF000C121F501C122F502C1AE
:1038B00023F503C124F50AEC37F038C5AFF539C557
:1038C000B0F53AC5B1F53BC5B2F53CC5B3F53DC55C
:1038D000B4F53EC5B5F5B7EC16F004012C0E826FB9
:1038E00093EC0EF03FC500F140C501F141C502F176
:1038F00042C503F10101000E046F000E056F010EB9
:10390000066F000E076F96EC2FF003EC30F029677E
:103910008CEF1CF091EF1CF004012D0E826F93ECE4
:103920000EF030C182F40401300E822793EC0EF0C9
:1039300031C182F40401300E822793EC0EF00401B1
:103940002E0E826F93EC0EF032C182F40401300E21
:10395000822793EC0EF033C182F40401300E8227EB
:1039600093EC0EF004012C0E826F93EC0EF060ECE1
:1039700030F043C500F144C501F1B5EC2AF0040173
:103980002C0E826F93EC0EF060EC30F045C500F128
:1039900003EC30F031C182F40401300E822793EC45
:1039A0000EF032C182F40401300E822793EC0EF047
:1039B00033C182F40401300E822793EC0EF004012F
:1039C0002C0E826F93EC0EF037C5E8FFE8B806D0F6
:1039D0000401300E826F93EC0EF005D00401310E1D
:1039E000826F93EC0EF007943FEF1EF0A1EC30F0E5
:1039F00085C32AF186C32BF187C32CF188C32DF12F
:103A000089C32EF18AC32FF18BC330F18CC331F1FE
:103A10008DC332F18EC333F10101296BAEEC30F06E
:103A200025EC30F00101010E046F000E056F000E51
:103A3000066F000E076F65EC2FF0100E046F000E7E
:103A4000056F000E066F000E076F76EC2FF000C1B9
:103A500029F501C12AF502C12BF503C12CF5DAECD9
:103A600034F004014C0E826F93EC0EF00401460E0C
:103A7000826F93EC0EF004012C0E826F93EC0EF02B
:103A800025C500F126C501F127C502F128C503F1BE
:103A90000101100E046F000E056F000E066F000E80
:103AA000076F96EC2FF003EC30F02AC182F404018A
:103AB000300E822793EC0EF02BC182F40401300EFD
:103AC000822793EC0EF02CC182F40401300E822781
:103AD00093EC0EF02DC182F40401300E822793EC9A
:103AE0000EF02EC182F40401300E822793EC0EF00A
:103AF0002FC182F40401300E822793EC0EF030C106
:103B000082F40401300E822793EC0EF031C182F46E
:103B10000401300E822793EC0EF032C182F40401CE
:103B2000300E822793EC0EF033C182F40401300E84
:103B3000822793EC0EF03FEF1EF037B0A2EF1DF09E
:103B4000020E166EB0EC35F000011650020AD8B421
:103B5000B9EF1DF015B2B4EF1DF081BAB4EF1DF04E
:103B6000000E166E8BEF29F0050E166E1584F9EF18
:103B700037F08B8001015E6B5F6B606B616B626B1A
:103B8000636B646B656B666B676B686B696B536BC0
:103B9000546BCF6ACE6A0F9A0F9C0F9E030E166E5F
:103BA0008BEF29F0B0EC35F015B2DEEF1DF081BAE5
:103BB000DEEF1DF0000E166E8BEF29F0050E166E6F
:103BC0001584F9EF37F004014C0E826F93EC0EF080
:103BD0000401350E826F93EC0EF004012C0E826FFF
:103BE00093EC0EF060EC30F00784B9C500F1079457
:103BF00003EC30F031C182F40401300E822793ECE3
:103C00000EF032C182F40401300E822793EC0EF0E4
:103C100033C182F40401300E822793EC0EF03FEFA3
:103C20001EF073EC35F060EC30F037C500F103ECBA
:103C300030F004014C0E826F93EC0EF00401360E4E
:103C4000826F93EC0EF004012C0E826F93EC0EF059
:103C500031C182F40401300E822793EC0EF032C1A0
:103C600082F40401300E822793EC0EF033C182F40B
:103C70000401300E822793EC0EF03FEF1EF09DEC16
:103C80000EF08BEF29F004014C0E826F93EC0EF0D6
:103C90000401500E826F93EC0EF004012C0E826F23
:103CA00093EC0EF085C32AF186C32BF187C32CF168
:103CB00088C32DF189C32EF18AC32FF18BC330F154
:103CC0008CC331F18DC332F18EC333F10101AEECFF
:103CD00030F025EC30F003018451530A0DE003016C
:103CE00084514D0A38E00401780E826F93EC0EF097
:103CF0009DEC0EF08BEF29F00401530E826F93ECD4
:103D00000EF0250E0C6E00C10BF04DEC0BF0260EE4
:103D10000C6E01C10BF04DEC0BF0270E0C6E02C1C6
:103D20000BF04DEC0BF0280E0C6E03C10BF04DECBC
:103D30000BF000C157F501C158F502C159F503C197
:103D40005AF500C15BF501C15CF502C15DF503C127
:103D50005EF520EF1FF004014D0E826F93EC0EF024
:103D6000290E0C6E00C10BF04DEC0BF000C15FF59D
:103D700000C160F520EF1FF004014C0E826F93EC40
:103D80000EF00401540E826F93EC0EF004012C0E21
:103D9000826F93EC0EF084C32AF185C32BF186C3A6
:103DA0002CF187C32DF188C32EF189C32FF18AC36B
:103DB00030F18BC331F18DC332F18EC333F1010188
:103DC000AEEC30F025EC30F00101000E046F000E77
:103DD000056F010E066F000E076F76EC2FF0210EB7
:103DE0000C6E00C10BF04DEC0BF0220E0C6E01C1FD
:103DF0000BF04DEC0BF0230E0C6E02C10BF04DECF2
:103E00000BF0240E0C6E03C10BF04DEC0BF000C157
:103E100061F501C162F502C163F503C164F520EFEC
:103E20001FF004014C0E826F93EC0EF00401490E5A
:103E3000826F93EC0EF004012C0E826F93EC0EF067
:103E4000250E64EC0BF0E8CF00F1260E64EC0BF0CD
:103E5000E8CF01F1270E64EC0BF0E8CF02F1280E59
:103E600064EC0BF0E8CF03F103EC30F0C6EC2DF07E
:103E70000401730E826F93EC0EF004012C0E826F1E
:103E800093EC0EF060EC30F0290E64EC0BF0E8CF10
:103E900000F103EC30F0C6EC2DF004016D0E826FE2
:103EA00093EC0EF004012C0E826F93EC0EF05BC5C8
:103EB00000F15CC501F15DC502F15EC503F103ECE3
:103EC00030F0C6EC2DF00401730E826F93EC0EF00F
:103ED00004012C0E826F93EC0EF060EC30F060C5A4
:103EE00000F103EC30F0C6EC2DF004016D0E826F92
:103EF00093EC0EF004012C0E826F93EC0EF061C572
:103F000000F162C501F163C502F164C503F1A6ECDD
:103F100029F004012C0E826F93EC0EF09DEC0EF054
:103F20008BEF29F083C32AF184C32BF185C32CF1D5
:103F300086C32DF187C32EF188C32FF189C330F1D9
:103F40008AC331F18BC332F18CC333F10101AEEC82
:103F500030F025EC30F0160E0C6E00C10BF04DEC7D
:103F60000BF0170E0C6E01C10BF04DEC0BF0180EA0
:103F70000C6E02C10BF04DEC0BF0190E0C6E03C170
:103F80000BF04DEC0BF000C18EF101C18FF102C1BD
:103F900090F103C191F100C192F101C193F102C10D
:103FA00094F103C195F174EF20F083C32AF184C327
:103FB0002BF185C32CF186C32DF187C32EF188C365
:103FC0002FF189C330F18AC331F18BC332F18CC335
:103FD00033F10101AEEC30F025EC30F000C18EF190
:103FE00001C18FF102C190F103C191F100C192F1C1
:103FF00001C193F102C194F103C195F174EF20F076
:1040000083C32AF184C32BF185C32CF186C32DF120
:1040100087C32EF188C32FF189C330F18AC331F1F0
:104020008CC332F18DC333F10101AEEC30F025ECDD
:1040300030F00101000E046F000E056F010E066FD7
:10404000000E076F76EC2FF01A0E0C6E00C10BF00D
:104050004DEC0BF01B0E0C6E01C10BF04DEC0BF098
:104060001C0E0C6E02C10BF04DEC0BF01D0E0C6E15
:1040700003C10BF04DEC0BF000C196F101C197F1BB
:1040800002C198F103C199F174EF20F083C32AF1C2
:1040900084C32BF185C32CF186C32DF187C32EF188
:1040A00088C32FF189C330F18AC331F18CC332F157
:1040B0008DC333F10101AEEC30F025EC30F001019D
:1040C000000E046F000E056F010E066F000E076FE5
:1040D00076EC2FF000C196F101C197F102C198F181
:1040E00003C199F174EF20F0160E64EC0BF0E8CFE9
:1040F00000F1170E64EC0BF0E8CF01F1180E64EC40
:104100000BF0E8CF02F1190E64EC0BF0E8CF03F1ED
:1041100003EC30F0C6EC2DF00401730E826F93ECCB
:104120000EF004012C0E826F93EC0EF08EC100F1A4
:104130008FC101F190C102F191C103F103EC30F0A4
:10414000C6EC2DF00401730E826F93EC0EF00401A7
:104150002C0E826F93EC0EF01A0E64EC0BF0E8CF8D
:1041600000F11B0E64EC0BF0E8CF01F11C0E64ECC7
:104170000BF0E8CF02F11D0E64EC0BF0E8CF03F179
:10418000A6EC29F004012C0E826F93EC0EF096C180
:1041900000F197C101F198C102F199C103F1A6ECB8
:1041A00029F09DEC0EF08BEF29F00401690E826F6F
:1041B00093EC0EF004012C0E826F93EC0EF00101D3
:1041C000040E006F000E016F000E026F000E036FF1
:1041D00003EC30F02CC182F40401300E822793EC02
:1041E0000EF02DC182F40401300E822793EC0EF004
:1041F0002EC182F40401300E822793EC0EF02FC101
:1042000082F40401300E822793EC0EF030C182F468
:104210000401300E822793EC0EF031C182F40401C8
:10422000300E822793EC0EF032C182F40401300E7E
:10423000822793EC0EF033C182F40401300E822702
:1042400093EC0EF004012C0E826F93EC0EF0010142
:10425000060E006F000E016F000E026F000E036F5E
:1042600003EC30F02CC182F40401300E822793EC71
:104270000EF02DC182F40401300E822793EC0EF073
:104280002EC182F40401300E822793EC0EF02FC170
:1042900082F40401300E822793EC0EF030C182F4D8
:1042A0000401300E822793EC0EF031C182F4040138
:1042B000300E822793EC0EF032C182F40401300EEE
:1042C000822793EC0EF033C182F40401300E822772
:1042D00093EC0EF004012C0E826F93EC0EF00101B2
:1042E000440E006F000E016F000E026F000E036F90
:1042F00003EC30F02CC182F40401300E822793ECE1
:104300000EF02DC182F40401300E822793EC0EF0E2
:104310002EC182F40401300E822793EC0EF02FC1DF
:1043200082F40401300E822793EC0EF030C182F447
:104330000401300E822793EC0EF031C182F40401A7
:10434000300E822793EC0EF032C182F40401300E5D
:10435000822793EC0EF033C182F40401300E8227E1
:1043600093EC0EF004012C0E826F93EC0EF0200EF5
:10437000F86EF76AF66A04010900F5CF82F493EC4F
:104380000EF00900F5CF82F493EC0EF00900F5CFA2
:1043900082F493EC0EF00900F5CF82F493EC0EF06A
:1043A0000900F5CF82F493EC0EF00900F5CF82F40A
:1043B00093EC0EF00900F5CF82F493EC0EF00900B7
:1043C000F5CF82F493EC0EF09DEC0EF08BEF29F01C
:1043D0008351630AD8A489EF29F08451610AD8A4D3
:1043E00089EF29F085516C0AD8A489EF29F086510C
:1043F000410A3FE08651440A1BE08651420AD8B484
:104400004CEF22F08651350AD8B415EF2BF08651C7
:10441000360AD8B46AEF2BF08651370AD8B4D3EFF6
:104420002BF08651380AD8B431EF2CF089EF29F0FF
:104430000798079A04017A0E826F93EC0EF004013C
:10444000780E826F93EC0EF00401640E826F93EC91
:104450000EF00401550E826F93EC0EF035EF22F052
:1044600004014C0E826F93EC0EF09DEC0EF08BEF7E
:1044700029F00788079A04017A0E826F93EC0EF0F8
:104480000401410E826F93EC0EF00401610E826F05
:1044900093EC0EF029EF22F00798078A04017A0EB8
:1044A000826F93EC0EF00401420E826F93EC0EF0DB
:1044B0000401610E826F93EC0EF029EF22F00101EE
:1044C00066676AEF22F067676AEF22F068676AEF53
:1044D00022F0696716D001014F6776EF22F050672E
:1044E00076EF22F0516776EF22F052670AD0010191
:1044F000000E006F000E016F000E026F000E036FC2
:10450000120011B80AD00101620E046F010E056F8E
:10451000000E066F000E076F09D00101A70E046F91
:10452000020E056F000E066F000E076F66C100F1E8
:1045300067C101F168C102F169C103F165EC2FF0B7
:1045400003BF13EF23F0119A119C0101000E046FB9
:10455000A80E056F550E066F020E076F66C100F1BB
:1045600067C101F168C102F169C103F166C18AF155
:1045700067C18BF168C18CF169C18DF165EC2FF0D9
:1045800003BF0BD00101000E8A6FA80E8B6F550E72
:104590008C6F020E8D6F118A119C0E0E64EC0BF065
:1045A000E8CF18F10F0E64EC0BF0E8CF19F1100E04
:1045B00064EC0BF0E8CF1AF1110E64EC0BF0E8CFCD
:1045C0001BF1AEEC2EF08AC104F18BC105F18CC158
:1045D00006F18DC107F165EC2FF0078272EC2EF029
:1045E000AEEC2EF0079272EC2EF08AC100F18BC176
:1045F00001F18CC102F18DC103F1079272EC2EF032
:10460000CC0E046FE00E056F870E066F050E076F68
:1046100065EC2FF000C118F101C119F102C11AF1C6
:1046200003C11BF140D013AA18EF23F0138E139A85
:10463000119C119A0101800E006F1A0E016F060E77
:10464000026F000E036F4FC104F150C105F151C15B
:1046500006F152C107F165EC2FF003AF05D060EC15
:1046600030F0118C119A12000E0E64EC0BF0E8CFB2
:1046700018F10F0E64EC0BF0E8CF19F1100E64EC9A
:104680000BF0E8CF1AF1110E64EC0BF0E8CF1BF140
:104690004FC100F150C101F151C102F152C103F10A
:1046A000078272EC2EF018C100F119C101F11AC194
:1046B00002F11BC103F112000784BAC166F1BBC14C
:1046C00067F1BCC168F1BDC169F14BC14FF14CC18B
:1046D00050F14DC151F14EC152F157C159F158C17C
:1046E0005AF10794010166677DEF23F067677DEF5C
:1046F00023F068677DEF23F0696716D001014F67EB
:1047000089EF23F0506789EF23F0516789EF23F099
:1047100052670AD00101000E006F000E016F000EFB
:10472000026F000E036F120011B80AD00101620E71
:10473000046F010E056F000E066F000E076F09D0A3
:104740000101A70E046F020E056F000E066F000E2A
:10475000076F66C100F167C101F168C102F169C16B
:1047600003F165EC2FF003BF15EF24F00101000EFB
:10477000046FA80E056F550E066F020E076F66C117
:1047800000F167C101F168C102F169C103F166C1BD
:104790008AF167C18BF168C18CF169C18DF165EC5B
:1047A0002FF003BF09D00101000E8A6FA80E8B6F96
:1047B000550E8C6F020E8D6FAEEC2EF000C104F121
:1047C00001C105F102C106F103C107F1000E006F3E
:1047D000A00E016F980E026F7B0E036F96EC2FF008
:1047E00000C118F101C119F102C11AF103C11BF195
:1047F000000E006FA00E016F980E026F7B0E036F0C
:104800008AC104F18BC105F18CC106F18DC107F19C
:1048100096EC2FF018C104F119C105F11AC106F187
:104820001BC107F165EC2FF012000101A80E006F0B
:10483000610E016F000E026F000E036F4FC104F195
:1048400050C105F151C106F152C107F165EC2FF0DD
:1048500003AF0AD00101A80E006F610E016F000EB8
:10486000026F000E036F00D0C80E006FAF0E016F15
:10487000000E026F000E036F4FC104F150C105F12D
:1048800051C106F152C107F176EC2FF0120004017C
:10489000730E826F93EC0EF004012C0E826F93EC7A
:1048A0000EF0078462C166F163C167F164C168F10B
:1048B00065C169F14BC14FF14CC150F14DC151F18E
:1048C0004EC152F157C159F158C15AF107946DECDC
:1048D00024F09DEC0EF08BEF29F066C100F167C16A
:1048E00001F168C102F169C103F1010103EC30F08B
:1048F000C6EC2DF00401630E826F93EC0EF0040100
:104900002C0E826F93EC0EF04FC100F150C101F1FB
:1049100051C102F152C103F1010103EC30F0C6ECC8
:104920002DF00401660E826F93EC0EF004012C0E44
:10493000826F93EC0EF060EC30F059C100F15AC177
:1049400001F1010103EC30F0C6EC2DF00401740E0E
:10495000826F93EC0EF0120010820401530E826FEE
:1049600093EC0EF004012C0E826F93EC0EF083C3D7
:104970002AF184C32BF185C32CF186C32DF187C3A3
:104980002EF188C32FF189C330F18AC331F18BC373
:1049900032F18CC333F10101AEEC30F025EC30F094
:1049A00000C166F101C167F102C168F103C169F19B
:1049B0008EC32AF18FC32BF190C32CF191C32DF13B
:1049C00092C32EF193C32FF194C330F195C331F10B
:1049D00096C332F197C333F10101AEEC30F025EC10
:1049E00030F000C14FF101C150F102C151F103C1DA
:1049F00052F1A1EC30F099C32FF19AC330F19BC36F
:104A000031F19CC332F19DC333F10101AEEC30F0C2
:104A100025EC30F000C159F101C15AF16DEC24F0E0
:104A200004012C0E826F93EC0EF027EF25F0118E0F
:104A30001CA002D01CAE108C1BBE02D01BA4108E7A
:104A400003018251520A02E10F8201D00F9282517A
:104A5000750A02E1108401D010948251550A02E1D6
:104A6000108601D010968351310A03E1138213841A
:104A700002D01392139403018351660A01E056D0C9
:104A80000401660E826F93EC0EF004012C0E826F0F
:104A900093EC0EF05CEC23F003EC30F02AC182F4CE
:104AA0000401300E822793EC0EF02BC182F4040136
:104AB000300E822793EC0EF02CC182F40401300EEC
:104AC000822793EC0EF02DC182F40401300E822770
:104AD00093EC0EF02EC182F40401300E822793EC89
:104AE0000EF02FC182F40401300E822793EC0EF0F9
:104AF00030C182F40401300E822793EC0EF031C1F4
:104B000082F40401300E822793EC0EF032C182F45D
:104B10000401300E822793EC0EF033C182F40401BD
:104B2000300E822793EC0EF089EF29F011A003D00C
:104B300011A401D01084078410B200EF26F010A455
:104B4000E4EF25F0BAC166F1BBC167F1BCC168F101
:104B5000BDC169F1BEC16AF1BFC16BF1C0C16CF1E9
:104B6000C1C16DF1C2C16EF1C3C16FF1C4C170F1B9
:104B7000C5C171F1C6C172F1C7C173F1C8C174F189
:104B8000C9C175F1CAC176F1CBC177F1CCC178F159
:104B9000CDC179F1CEC17AF1CFC17BF1D0C17CF129
:104BA000D1C17DF1D2C17EF1D3C17FF1D4C180F1F9
:104BB000D5C181F1D6C182F1D7C183F1D8C184F1C9
:104BC000D9C185F1ECEF25F062C166F163C167F1EF
:104BD00064C168F165C169F1BAC186F1BBC187F1F1
:104BE000BCC188F1BDC189F14BC14FF14CC150F13D
:104BF0004DC151F14EC152F157C159F158C15AF14D
:104C000007940FA022EF26F0010196670FEF26F020
:104C100097670FEF26F098670FEF26F0996713EF6D
:104C200026F022EF26F05FEC22F096C104F197C146
:104C300005F198C106F199C107F165EC2FF003BFAA
:104C40004FEF29F05FEC22F00101000E046F000E1F
:104C5000056F010E066F000E076F96EC2FF011A086
:104C60002AD011A228D003EC30F0296701D005D05A
:104C700004012D0E826F93EC0EF030C182F404011A
:104C8000300E822793EC0EF031C182F40401300E15
:104C9000822793EC0EF032C182F40401300E822799
:104CA00093EC0EF033C182F40401300E822793ECB2
:104CB0000EF09DEC0EF012A8C5D012981DC01EF08B
:104CC0001E3A1E42070E1E1600011E50000AD8B4DE
:104CD000EEEF26F000011E50010AD8B47AEF26F05C
:104CE00000011E50020AD8B478EF26F020EF27F01A
:104CF00020EF27F060EC30F02DC001F12EC000F164
:104D0000D89001330033D890013300330101630E92
:104D1000046F000E056F000E066F000E076F96EC15
:104D20002FF0280E046F000E056F000E066F000EA8
:104D3000076F65EC2FF000C130F060EC30F02BC055
:104D400001F1019F019D2CC000F10101A40E046F2F
:104D5000000E056F000E066F000E076F96EC2FF029
:104D600000C12FF000C104F101C105F102C106F13B
:104D700003C107F1640E006F000E016F000E026F99
:104D8000000E036F65EC2FF0050E046F000E056F2B
:104D9000000E066F000E076F96EC2FF000C104F1B5
:104DA00001C105F102C106F103C107F160EC30F069
:104DB00030C000F165EC2FF000C131F031C0E8FFE8
:104DC000050F305C03E78A8420EF27F031C0E8FF4D
:104DD0000A0F305C01E68A9420EF27F000C124F12D
:104DE00001C125F102C126F103C127F160EC30F0C9
:104DF00066EC30F01D501F0BE8CF00F10101640E8E
:104E0000046F000E056F000E066F000E076F76EC44
:104E10002FF024C104F125C105F126C106F127C1F7
:104E200007F165EC2FF003BF02D08A9401D08A8489
:104E300024C100F125C101F126C102F127C103F10E
:104E40008BEF29F000C124F101C125F102C126F147
:104E500003C127F110AE4DD0109E00C108F101C171
:104E600009F102C10AF103C10BF103EC30F030C1CA
:104E7000E2F131C1E3F132C1E4F133C1E5F108C13E
:104E800000F109C101F10AC102F10BC103F10101F5
:104E90006C0E046F070E056F000E066F000E076F95
:104EA00065EC2FF003BF04D00101550EE66F1CD056
:104EB00008C100F109C101F10AC102F10BC103F1FE
:104EC0000101A40E046F060E056F000E066F000EA2
:104ED000076F65EC2FF003BF04D001017F0EE66F72
:104EE00003D00101FF0EE66F1F8E11AE4FEF29F0C8
:104EF000119E24C100F125C101F126C102F127C193
:104F000003F111A005D011A203D00FB04FEF29F08B
:104F100010A492EF27F00401750E826F93EC0EF04F
:104F200097EF27F00401720E826F93EC0EF00401EC
:104F30002C0E826F93EC0EF003EC30F02967A6EF95
:104F400027F00401200E826FA9EF27F004012D0E37
:104F5000826F93EC0EF030C182F40401300E822790
:104F600093EC0EF031C182F40401300E822793ECF1
:104F70000EF004012E0E826F93EC0EF032C182F41B
:104F80000401300E822793EC0EF033C182F4040149
:104F9000300E822793EC0EF004016D0E826F93ECBD
:104FA0000EF004012C0E826F93EC0EF04FC100F155
:104FB00050C101F151C102F152C103F1010103ECF1
:104FC00030F0C6EC2DF00401480E826F93EC0EF029
:104FD00004017A0E826F93EC0EF004012C0E826FA6
:104FE00093EC0EF066C100F167C101F168C102F1F6
:104FF00069C103F1010103EC30F0C6EC2DF00401AE
:10500000630E826F93EC0EF004012C0E826F93EC12
:105010000EF066C100F167C101F168C102F169C11A
:1050200003F101010A0E046F000E056F000E066FFA
:10503000000E076F76EC2FF0000E046F120E056F56
:10504000000E066F000E076F96EC2FF003EC30F0A9
:105050002AC182F40401300E822793EC0EF02BC19A
:1050600082F40401300E822793EC0EF02CC182F4FE
:105070000401300E822793EC0EF02DC182F404015E
:10508000300E822793EC0EF02EC182F40401300E14
:10509000822793EC0EF02FC182F40401300E822798
:1050A00093EC0EF030C182F40401300E822793ECB1
:1050B0000EF004012E0E826F93EC0EF031C182F4DB
:1050C0000401300E822793EC0EF032C182F4040109
:1050D000300E822793EC0EF033C182F40401300EBF
:1050E000822793EC0EF00401730E826F93EC0EF0A6
:1050F00004012C0E826F93EC0EF060EC30F059C17D
:1051000000F15AC101F1B5EC2AF013A2D7EF28F053
:1051100004012C0E826F93EC0EF086C166F187C1FC
:1051200067F188C168F189C169F15FEC22F0010182
:10513000000E046F000E056F010E066F000E076F64
:1051400096EC2FF003EC30F02967ACEF28F0040167
:10515000200E826FAFEF28F004012D0E826F93ECCA
:105160000EF030C182F40401300E822793EC0EF071
:1051700031C182F40401300E822793EC0EF0040159
:105180002E0E826F93EC0EF032C182F40401300EC9
:10519000822793EC0EF033C182F40401300E822793
:1051A00093EC0EF004016D0E826F93EC0EF013A4DD
:1051B000FEEF28F004012C0E826F93EC0EF013AC7E
:1051C000ECEF28F00401500E826F93EC0EF0139C6C
:1051D0001398139AFEEF28F013AEF9EF28F00401AC
:1051E000460E826F93EC0EF0139E1398139AFEEF07
:1051F00028F00401530E826F93EC0EF037B015EFD8
:1052000029F004012C0E826F93EC0EF08BB010EF9E
:1052100029F00401440E826F93EC0EF015EF29F093
:105220000401530E826F93EC0EF00FB21BEF29F0C6
:105230000FA04DEF29F004012C0E826F93EC0EF0BD
:10524000200EF86EF76AF66A04010900F5CF82F4C1
:1052500093EC0EF00900F5CF82F493EC0EF0090008
:10526000F5CF82F493EC0EF00900F5CF82F493ECC5
:105270000EF00900F5CF82F493EC0EF00900F5CFA3
:1052800082F493EC0EF00900F5CF82F493EC0EF06B
:105290000900F5CF82F493EC0EF09DEC0EF00F9028
:1052A000109E12988BEF29F00401630E826F93EC2D
:1052B0000EF004012C0E826F93EC0EF091EC29F0AD
:1052C00004012C0E826F93EC0EF004EC2AF0040122
:1052D0002C0E826F93EC0EF080EC2AF004012C0E61
:1052E000826F93EC0EF00101F80E006FCD0E016F8E
:1052F000660E026F030E036FA6EC29F004012C0E5C
:10530000826F93EC0EF096EC2AF09DEC0EF08BEF92
:1053100029F09DEC0EF00301C26B079010929AEFFA
:105320002CF0D8900E0E64EC0BF0E8CF00F10F0ECD
:1053300064EC0BF0E8CF01F1100E64EC0BF0E8CF59
:1053400002F1110E64EC0BF0E8CF03F10101000E45
:10535000046F000E056F010E066F000E076F96ECCE
:105360002FF003EC30F02AC182F40401300E8227C2
:1053700093EC0EF02BC182F40401300E822793ECE3
:105380000EF02CC182F40401300E822793EC0EF053
:105390002DC182F40401300E822793EC0EF02EC151
:1053A00082F40401300E822793EC0EF02FC182F4B8
:1053B0000401300E822793EC0EF030C182F4040118
:1053C000300E822793EC0EF031C182F40401300ECE
:1053D000822793EC0EF004012E0E826F93EC0EF0F8
:1053E00032C182F40401300E822793EC0EF033C1F7
:1053F00082F40401300E822793EC0EF004016D0E4E
:10540000826F93EC0EF01200120E64EC0BF0E8CFFA
:1054100000F1130E64EC0BF0E8CF01F1140E64EC14
:105420000BF0E8CF02F1150E64EC0BF0E8CF03F1BE
:1054300001010A0E046F000E056F000E066F000ECC
:10544000076F76EC2FF0000E046F120E056F000E42
:10545000066F000E076F96EC2FF003EC30F02AC1B8
:1054600082F40401300E822793EC0EF02BC182F4FB
:105470000401300E822793EC0EF02CC182F404015B
:10548000300E822793EC0EF02DC182F40401300E11
:10549000822793EC0EF02EC182F40401300E822795
:1054A00093EC0EF02FC182F40401300E822793ECAE
:1054B0000EF030C182F40401300E822793EC0EF01E
:1054C00004012E0E826F93EC0EF031C182F40401C0
:1054D000300E822793EC0EF032C182F40401300EBC
:1054E000822793EC0EF033C182F40401300E822740
:1054F00093EC0EF00401730E826F93EC0EF0120029
:105500000A0E64EC0BF0E8CF00F10B0E64EC0BF02C
:10551000E8CF01F10C0E64EC0BF0E8CF02F10D0EB8
:1055200064EC0BF0E8CF03F1B5EF2AF0060E64EC63
:105530000BF0E8CF00F1070E64EC0BF0E8CF01F1BF
:10554000080E64EC0BF0E8CF02F1090E64EC0BF0EE
:10555000E8CF03F1B5EF2AF0010160EC30F00784E9
:1055600057C100F158C101F107940101E80E046F21
:10557000800E056F000E066F000E076F76EC2FF0A1
:10558000000E046F040E056F000E066F000E076F0D
:1055900096EC2FF0880E046F130E056F000E066F49
:1055A000000E076F65EC2FF00A0E046F000E056FFA
:1055B000000E066F000E076F96EC2FF003EC30F034
:1055C00001012967E9EF2AF00401200E826FECEF58
:1055D0002AF004012D0E826F93EC0EF030C182F49C
:1055E0000401300E822793EC0EF031C182F40401E5
:1055F000300E822793EC0EF032C182F40401300E9B
:10560000822793EC0EF004012E0E826F93EC0EF0C5
:1056100033C182F40401300E822793EC0EF00401B2
:10562000430E826F93EC0EF0120087C32AF188C3F9
:105630002BF189C32CF18AC32DF18BC32EF18CC3BE
:105640002FF18DC330F18EC331F190C332F191C38C
:1056500033F10101296BAEEC30F025EC30F00101A3
:10566000000E046F000E056F010E066F000E076F2F
:1056700076EC2FF00E0E0C6E00C10BF04DEC0BF023
:105680000F0E0C6E01C10BF04DEC0BF0100E0C6EFA
:1056900002C10BF04DEC0BF0110E0C6E03C10BF0C0
:1056A0004DEC0BF004017A0E826F93EC0EF00401C6
:1056B0002C0E826F93EC0EF00401350E826F93EC8A
:1056C0000EF004012C0E826F93EC0EF091EC29F099
:1056D00035EF22F087C32AF188C32BF189C32CF15F
:1056E0008AC32DF18BC32EF18CC32FF18DC330F102
:1056F0008EC331F190C332F191C333F10101296BB3
:10570000AEEC30F025EC30F0880E046F130E056F10
:10571000000E066F000E076F6AEC2FF0000E046F8C
:10572000040E056F000E066F000E076F76EC2FF06B
:105730000101E80E046F800E056F000E066F000E6B
:10574000076F96EC2FF00A0E0C6E00C10BF04DECBB
:105750000BF00B0E0C6E01C10BF04DEC0BF00C0EB0
:105760000C6E02C10BF04DEC0BF00D0E0C6E03C174
:105770000BF04DEC0BF004017A0E826F93EC0EF0FF
:1057800004012C0E826F93EC0EF00401360E826F32
:1057900093EC0EF004012C0E826F93EC0EF080EC73
:1057A0002AF035EF22F087C32AF188C32BF189C391
:1057B0002CF18AC32DF18BC32EF18CC32FF18DC335
:1057C00030F18FC331F190C332F191C333F1010154
:1057D000AEEC30F025EC30F0000E046F120E056FC9
:1057E000000E066F000E076F76EC2FF001010A0E17
:1057F000046F000E056F000E066F000E076F96EC2B
:105800002FF0120E0C6E00C10BF04DEC0BF0130ECE
:105810000C6E01C10BF04DEC0BF0140E0C6E02C1BE
:105820000BF04DEC0BF0150E0C6E03C10BF04DECB4
:105830000BF004017A0E826F93EC0EF004012C0E33
:10584000826F93EC0EF00401370E826F93EC0EF032
:1058500004012C0E826F93EC0EF004EC2AF035EF6D
:1058600022F087C32AF188C32BF189C32CF18AC3A4
:105870002DF18BC32EF18CC32FF18DC330F18EC36C
:1058800031F190C332F191C333F10101296BAEECD8
:1058900030F025EC30F0880E046F130E056F000E0B
:1058A000066F000E076F6AEC2FF0000E046F040EF7
:1058B000056F000E066F000E076F76EC2FF00101EA
:1058C000E80E046F800E056F000E066F000E076F66
:1058D00096EC2FF0060E0C6E00C10BF04DEC0BF0A9
:1058E000070E0C6E01C10BF04DEC0BF0080E0C6EA8
:1058F00002C10BF04DEC0BF0090E0C6E03C10BF066
:105900004DEC0BF004017A0E826F93EC0EF0040163
:105910002C0E826F93EC0EF00401380E826F93EC24
:105920000EF004012C0E826F93EC0EF096EC2AF030
:1059300035EF22F007A80DEF2DF00101800E006F6A
:105940001A0E016F060E026F000E036F4BC104F1B9
:105950004CC105F14DC106F14EC107F165EC2FF0C8
:1059600003BF53EF2DF0C0EC2DF04BC100F14CC143
:1059700001F14DC102F14EC103F1078272EC2EF02C
:1059800018C104F119C105F11AC106F11BC107F1D3
:10599000F80E006FCD0E016F660E026F030E036FDF
:1059A00065EC2FF00E0E0C6E00C10BF04DEC0BF001
:1059B0000F0E0C6E01C10BF04DEC0BF0100E0C6EC7
:1059C00002C10BF04DEC0BF0110E0C6E03C10BF08D
:1059D0004DEC0BF00784010160EC30F057C100F191
:1059E00058C101F107940A0E0C6E00C10BF04DEC8A
:1059F0000BF00B0E0C6E01C10BF04DEC0BF00C0E0E
:105A00000C6E02C10BF04DEC0BF00D0E0C6E03C1D1
:105A10000BF04DEC0BF053EF2DF007AA53EF2DF0E8
:105A20000784010160EC30F057C100F158C101F169
:105A30000794060E0C6E00C10BF04DEC0BF0070E38
:105A40000C6E01C10BF04DEC0BF0080E0C6E02C198
:105A50000BF04DEC0BF0090E0C6E03C10BF04DEC8E
:105A60000BF0078462C100F163C101F164C102F16E
:105A700065C103F10794120E0C6E00C10BF04DECE2
:105A80000BF0130E0C6E01C10BF04DEC0BF0140E6D
:105A90000C6E02C10BF04DEC0BF0150E0C6E03C139
:105AA0000BF04DEC0BF00798079A04018051811917
:105AB0007F0B0DE09EA8FED714EE00F081517F0B06
:105AC000E126E750812B0F01AD6E55EF2DF005015A
:105AD0002F51010A14E081BA73EF2DF015B288EF4F
:105AE0002DF07FEF2DF005012F51000AD8B4F9EF0A
:105AF00037F000011650050AD8B4F9EF37F081B835
:105B000088EF2DF0A9EC31F0A7EC32F096EC37F0ED
:105B1000C1EF0DF018C100F119C101F11AC102F174
:105B20001BC103F1000E046F000E056F010E066F1E
:105B3000000E076F96EC2FF029A1B5EF2DF0205144
:105B4000D8B4B5EF2DF018C100F119C101F11AC197
:105B500002F11BC103F1000E046F000E056F0A0E67
:105B6000066F000E076F96EC2FF012000101045132
:105B700000130551011306510213075103131200BC
:105B80000101186B196B1A6B1B6B12002AC182F48E
:105B90000401300E822793EC0EF02BC182F4040135
:105BA000300E822793EC0EF02CC182F40401300EEB
:105BB000822793EC0EF02DC182F40401300E82276F
:105BC00093EC0EF02EC182F40401300E822793EC88
:105BD0000EF02FC182F40401300E822793EC0EF0F8
:105BE00030C182F40401300E822793EC0EF031C1F3
:105BF00082F40401300E822793EC0EF032C182F45D
:105C00000401300E822793EC0EF033C182F40401BC
:105C1000300E822793EC0EF012002FC182F40401A3
:105C2000300E822793EC0EF030C182F40401300E66
:105C3000822793EC0EF031C182F40401300E8227EA
:105C400093EC0EF032C182F40401300E822793EC03
:105C50000EF033C182F40401300E822793EC0EF073
:105C60001200060E216E060E226E060E236E212EE7
:105C700037EF2EF0222E37EF2EF0232E37EF2EF0B7
:105C80008B84020E216E020E226E020E236E212ED6
:105C900047EF2EF0222E47EF2EF0232E47EF2EF067
:105CA0008B941200FF0E226E22C023F0030E216E91
:105CB0008B84212E58EF2EF0030E216E232E58EFE9
:105CC0002EF08B9422C023F0030E216E212E66EF5E
:105CD0002EF0030E216E233E66EF2EF0222E54EF9F
:105CE0002EF012000101005305E1015303E10253BC
:105CF00001E1002B35EC2FF060EC30F03951006FF2
:105D00003A51016F420E046F4B0E056F000E066F85
:105D1000000E076F76EC2FF000C104F101C105F110
:105D200002C106F103C107F118C100F119C101F167
:105D30001AC102F11BC103F107B2A3EF2EF06AEC06
:105D40002FF0A5EF2EF065EC2FF000C118F101C186
:105D500019F102C11AF103C11BF1120060EC30F01D
:105D600059C100F15AC101F1060E64EC0BF0E8CF05
:105D700004F1070E64EC0BF0E8CF05F1080E64ECBB
:105D80000BF0E8CF06F1090E64EC0BF0E8CF07F159
:105D900065EC2FF000C124F101C125F102C126F10B
:105DA00003C127F1290E046F000E056F000E066F68
:105DB000000E076F76EC2FF0EE0E046F430E056FAA
:105DC000000E066F000E076F6AEC2FF024C104F17D
:105DD00025C105F126C106F127C107F176EC2FF0A8
:105DE00000C11CF101C11DF102C11EF103C11FF16F
:105DF000120E64EC0BF0E8CF04F1130E64EC0BF020
:105E0000E8CF05F1140E64EC0BF0E8CF06F1150EA7
:105E100064EC0BF0E8CF07F10D0E006F000E016F80
:105E2000000E026F000E036F76EC2FF0180E046F59
:105E3000000E056F000E066F000E076F96EC2FF038
:105E40001CC104F11DC105F11EC106F11FC107F1FE
:105E50006AEC2FF06A0E046F2A0E056F000E066FB3
:105E6000000E076F65EC2FF01200BF0EFA6E200EC9
:105E70003A6F396BD8900037013702370337D8B003
:105E800046EF2FF03A2F3BEF2FF039073A07035335
:105E9000D8B412000331070B80093F6F03390F0B91
:105EA000010F396F80EC5FF0406F390580EC5FF0D7
:105EB000405D405F396B3F33D8B0392739333FA954
:105EC0005BEF2FF0405139271200010185EC30F0D3
:105ED000D8B01200010103510719346F48EC30F0BB
:105EE000D8900751031934AF800F12000101346BB1
:105EF0006CEC30F0D8A082EC30F0D8B0120057EC47
:105F000030F060EC30F01F0E366F98EC30F00B354F
:105F1000D8B048EC30F0D8A00335D8B01200362FF6
:105F200085EF2FF034B16FEC30F012000101346BCB
:105F300004510511061107110008D8A06CEC30F0CF
:105F4000D8A082EC30F0D8B01200086B096B0A6B55
:105F50000B6B98EC30F01F0E366F98EC30F0075159
:105F60000B5DD8A4C0EF2FF006510A5DD8A4C0EF96
:105F70002FF00551095DD8A4C0EF2FF00451085D42
:105F8000D8A0D3EF2FF00451085F0551D8A0053DEC
:105F9000095F0651D8A0063D0A5F0751D8A0073D0A
:105FA0000B5FD8900081362FADEF2FF034B16FEC3E
:105FB00030F0346B6CEC30F0D8909CEC30F0075142
:105FC0000B5DD8A4F0EF2FF006510A5DD8A4F0EFD6
:105FD0002FF00551095DD8A4F0EF2FF00451085DB2
:105FE000D8A0FFEF2FF0003FFFEF2FF0013FFFEFB2
:105FF0002FF0023FFFEF2FF0032BD8B4120034B183
:106000006FEC30F012000101346B6CEC30F0D8B062
:106010001200A1EC30F0200E366F00370137023746
:10602000033711EE33F00A0E376FE7360A0EE75CDE
:10603000D8B0E76EE552372F15EF30F0362F0DEF61
:1060400030F034B12981D890120001010A0E346F6A
:10605000200E366F11EE29F03451376F0A0ED890AA
:10606000E652D8B0E726E732372F30EF30F003336F
:10607000023301330033362F2AEF30F0E750FF0FA1
:10608000D8A00335D8B0120029B16FEC30F012005F
:10609000045100270551D8B0053D01270651D8B05D
:1060A000063D02270751D8B0073D032712000051D3
:1060B000086F0151096F02510A6F03510B6F1200F3
:1060C0000101006B016B026B036B12000101046B99
:1060D000056B066B076B12000335D8A01200035145
:1060E000800B001F011F021F031F003F7FEF30F0D6
:1060F000013F7FEF30F0023F7FEF30F0032B342B76
:10610000032512000735D8A012000751800B041F89
:10611000051F061F071F043F95EF30F0053F95EF61
:1061200030F0063F95EF30F0072B342B0725120097
:106130000037013702370337083709370A370B377B
:1061400012000101296B2A6B2B6B2C6B2D6B2E6BB4
:106150002F6B306B316B326B336B120001012A51A4
:106160000F0B2A6F2B510F0B2B6F2C510F0B2C6F1A
:106170002D510F0B2D6F2E510F0B2E6F2F510F0B1B
:106180002F6F30510F0B306F31510F0B316F325178
:106190000F0B326F33510F0B336F120000C124F11C
:1061A00001C125F102C126F103C127F104C100F1AB
:1061B00005C101F106C102F107C103F124C104F1D7
:1061C00025C105F126C106F127C107F1120010A86B
:1061D00006D08994000EC76E220EC66E05D0898443
:1061E000000EC76E220EC66E050EE82EFED71200F8
:1061F00010A802D0898401D08994050EE82EFED71C
:106200001200E7EC30F09E96C69E000EC96EFF0E9F
:106210009EB602D0E82EFCD79E96C69E000EC96E92
:10622000FF0E9EB602D0E82EFCD7C9CFAFF59E96E2
:10623000C69E000EC96EFF0E9EB602D0E82EFCD799
:10624000C9CFB0F59E96C69E000EC96EFF0E9EB6D3
:1062500002D0E82EFCD7C9CFB1F59E96C69E000E9F
:10626000C96EFF0E9EB602D0E82EFCD7C9CFB2F59C
:106270009E96C69E000EC96EFF0E9EB602D0E82EF8
:10628000FCD7C9CFB3F59E96C69E000EC96EFF0E11
:106290009EB602D0E82EFCD7C9CFB4F59E96C69E16
:1062A000000EC96EFF0E9EB602D0E82EFCD7C9CFF5
:1062B000B5F5F8EC30F01200E7EC30F09E96C69E93
:1062C000800EC96EFF0E9EB602D0E82EFCD79E96B9
:1062D000C69EAFC5C9FFFF0E9EB602D0E82EFCD702
:1062E0009E96C69EB0C5C9FFFF0E9EB602D0E82E90
:1062F000FCD79E96C69EB1C5C9FFFF0E9EB602D0C2
:10630000E82EFCD79E96C69EB2C5C9FFFF0E9EB66C
:1063100002D0E82EFCD79E96C69EB3C5C9FFFF0EDD
:106320009EB602D0E82EFCD79E96C69EB4C5C9FF85
:10633000FF0E9EB602D0E82EFCD79E96C69EB5C52F
:10634000C9FFFF0E9EB602D0E82EFCD7F8EC30F065
:106350001200E7EC30F09E96C69E070EC96EFF0E47
:106360009EB602D0E82EFCD79E96C69E000EC96E41
:10637000FF0E9EB602D0E82EFCD7C9CFAFF59E9691
:10638000C69E000EC96EFF0E9EB602D0E82EFCD748
:10639000C9CFB0F59E96C69E000EC96EFF0E9EB682
:1063A00002D0E82EFCD7C9CFB1F59E96C69E000E4E
:1063B000C96EFF0E9EB602D0E82EFCD7C9CFB2F54B
:1063C000F8EC30F0E7EC30F09E96C69E25C0C9FF91
:1063D000FF0E9EB602D0E82EFCD79E96C69E000EFB
:1063E000C96EFF0E9EB602D0E82EFCD7C9CFB6F517
:1063F000F8EC30F01200E7EC30F09E96C69E870E67
:10640000C96EFF0E9EB602D0E82EFCD79E96C69EA1
:10641000AFC5C9FFFF0E9EB602D0E82EFCD79E96F0
:10642000C69EB0C5C9FFFF0E9EB602D0E82EFCD7AF
:106430009E96C69EB1C5C9FFFF0E9EB602D0E82E3D
:10644000FCD79E96C69EB2C5C9FFFF0E9EB602D06F
:10645000E82EFCD7F8EC30F0E7EC30F09E96C69EC4
:1064600026C0C9FFFF0E9EB602D0E82EFCD79E962E
:10647000C69EB6C5C9FFFF0E9EB602D0E82EFCD759
:10648000F8EC30F01200E7EC30F09E96C69E870ED6
:10649000C96EFF0E9EB602D0E82EFCD79E96C69E11
:1064A000000EC96EFF0E9EB602D0E82EFCD79E9657
:1064B000C69E800EC96EFF0E9EB602D0E82EFCD797
:1064C0009E96C69E800EC96EFF0E9EB602D0E82E26
:1064D000FCD79E96C69E800EC96EFF0E9EB602D059
:1064E000E82EFCD7F8EC30F01200E7EC30F09E9686
:1064F000C69E870EC96EFF0E9EB602D0E82EFCD750
:106500009E96C69E000EC96EFF0E9EB602D0E82E65
:10651000FCD79E96C69E000EC96EFF0E9EB602D098
:10652000E82EFCD79E96C69E800EC96EFF0E9EB6C4
:1065300002D0E82EFCD79E96C69E800EC96EFF0E36
:106540009EB602D0E82EFCD7F8EC30F0120010A86E
:1065500017D0E7EC30F09E96C69E8F0EC96EFF0EE8
:106560009EB602D0E82EFCD79E96C69E000EC96E3F
:10657000FF0E9EB602D0E82EFCD7F8EC30F01200E9
:10658000A9EC31F0120010A82DD0E7EC30F09E9667
:10659000C69E26C0C9FFFF0E9EB602D0E82EFCD7CD
:1065A0009E96C69E450EC96EFF0E9EB602D0E82E80
:1065B000FCD7F8EC30F0E7EC30F09E96C69E8F0EDC
:1065C000C96EFF0E9EB602D0E82EFCD79E96C69EE0
:1065D000000EC96EFF0E9EB602D0E82EFCD7F8EC76
:1065E00030F01200E7EC30F09E96C69E26C0C9FF40
:1065F000FF0E9EB602D0E82EFCD79E96C69E010ED8
:10660000C96EFF0E9EB602D0E82EFCD7F8EC30F033
:10661000E7EC30F09E96C69E910EC96EFF0E9EB6B8
:1066200002D0E82EFCD79E96C69EA50EC96EFF0E20
:106630009EB602D0E82EFCD7F8EC30F01200E7EC62
:1066400030F09E96C69E26C0C9FFFF0E9EB602D0B1
:10665000E82EFCD79E96C69E810EC96EFF0E9EB692
:1066600002D0E82EFCD7F8EC30F01200E7EC30F066
:106670009E96C69E26C0C9FFFF0E9EB602D0E82E8B
:10668000FCD79E96C69E010EC96EFF0E9EB602D026
:10669000E82EFCD7F8EC30F01200E7EC30F09E96D4
:1066A000C69E910EC96EFF0E9EB602D0E82EFCD794
:1066B0009E96C69EA50EC96EFF0E9EB602D0E82E0F
:1066C000FCD7F8EC30F01200E7EC30F09E96C69E56
:1066D000910EC96EFF0E9EB602D0E82EFCD79E9694
:1066E000C69E000EC96EFF0E9EB602D0E82EFCD7E5
:1066F000F8EC30F012000501256B266B276B286B38
:10670000899A400EC76E200EC66E9E96C69E030ED8
:10671000C96EFF0E9EB602D0E82EFCD79E96C69E8E
:1067200027C5C9FFFF0E9EB602D0E82EFCD79E9665
:10673000C69E26C5C9FFFF0E9EB602D0E82EFCD726
:106740009E96C69E25C5C9FFFF0E9EB602D0E82EB6
:10675000FCD79E96C69EC952FF0E9EB602D0E82E6A
:10676000FCD7898A0F01C950FF0A01E11200050117
:106770002E51130A05E005012E51170A0CE01200F4
:106780000501F00E256FFF0E266F0F0E276F000E0E
:10679000286FD4EF33F00501F00E256FFF0E266F42
:1067A000FF0E276F000E286F899A400EC76E200ECD
:1067B000C66E9E96C69E030EC96EFF0E9EB602D092
:1067C000E82EFCD79E96C69E27C5C9FFFF0E9EB633
:1067D00002D0E82EFCD79E96C69E26C5C9FFFF0EA6
:1067E0009EB602D0E82EFCD79E96C69E25C5C9FF50
:1067F000FF0E9EB602D0E82EFCD79E96C69EC952CA
:10680000FF0E9EB602D0E82EFCD7898A0F01C95030
:10681000FF0A1DE005012E51130A05E005012E5166
:10682000170A0BE012000501000E256F000E266FFF
:10683000100E276F000E286F12000501000E256F45
:10684000000E266F000E276F010E286F1200050143
:10685000256B266B276B286B05012E51130A05E06B
:1068600005012E51170A0CE012000501000E216FE0
:10687000000E226F080E236F000E246F49EF34F0D4
:106880000501000E216F000E226F800E236F000E97
:10689000246F21C500F122C501F123C502F124C5F1
:1068A00003F125C504F126C505F127C506F128C564
:1068B00007F1B6EC2DF000C125F501C126F502C1A6
:1068C00027F503C128F5899A400EC76E200EC66EC3
:1068D0009E96C69E030EC96EFF0E9EB602D0E82E8F
:1068E000FCD79E96C69E27C5C9FFFF0E9EB602D056
:1068F000E82EFCD79E96C69E26C5C9FFFF0E9EB603
:1069000002D0E82EFCD79E96C69E25C5C9FFFF0E75
:106910009EB602D0E82EFCD79E96C69EC952FF0EA8
:106920009EB602D0E82EFCD7898AC950FF0A08E13A
:1069300004C125F505C126F506C127F507C128F5CF
:10694000D890050124332333223321332151F00B16
:10695000216F05012167B4EF34F02267B4EF34F002
:106960002367B4EF34F0246749EF34F00501100ECB
:106970002527E86A2623E86A2723E86A28231200E5
:10698000E86A05012E51130A06E005012E51170A87
:106990000BE0020E120005012851000A03E1275105
:1069A000F00B07E0010E120005012851000A01E07A
:1069B000010E120029C500F12AC501F12BC502F113
:1069C0002CC503F125C504F126C505F127C506F13F
:1069D00028C507F165EC2FF003BF1200C0EC34F0BE
:1069E000D8A452EF35F0899A400EC76E200EC66EBD
:1069F0009E96C69E060EC96EFF0E9EB602D0E82E6B
:106A0000FCD7898A899A9E96C69E020EC96EFF0E91
:106A10009EB602D0E82EFCD79E96C69E27C5C9FF1B
:106A2000FF0E9EB602D0E82EFCD79E96C69E26C5C7
:106A3000C9FFFF0E9EB602D0E82EFCD79E96C69EDA
:106A400025C5C9FFFF0E9EB602D0E82EFCD79E9644
:106A5000C69E000EC96EFF0E9EB602D0E82EFCD771
:106A6000898A899A9E96C69E050EC96EFF0E9EB6AD
:106A700002D0E82EFCD79E96C69EC952FF0E9EB647
:106A800002D0E82EFCD7C9B03BEF35F0898A05016A
:106A9000100E2527E86A2623E86A2723E86A2823B8
:106AA000DAEF34F01200899A400EC76E200EC66EDF
:106AB0009E96C69E060EC96EFF0E9EB602D0E82EAA
:106AC000FCD7898A899A9E96C69EC70EC96EFF0E0C
:106AD0009EB602D0E82EFCD7898A0501256B266B6D
:106AE000276B286B1200899A400EC76E200EC66E67
:106AF0009E96C69E050EC96EFF0E9EB602D0E82E6B
:106B0000FCD79E96C69EC952FF0E9EB602D0E82EB6
:106B1000FCD7C9CF37F5898A1200899A400EC76E13
:106B2000200EC66E9E96C69EB90EC96EFF0E9EB60C
:106B300002D0E82EFCD7898A1200899A400EC76ECF
:106B4000200EC66E9E96C69EAB0EC96EFF0E9EB6FA
:106B500002D0E82EFCD7898AFF0EE82EFED712005D
:106B6000C0EC34F0D8A41200899A400EC76E200EF3
:106B7000C66E9E96C69E030EC96EFF0E9EB602D0CE
:106B8000E82EFCD79E96C69E27C5C9FFFF0E9EB66F
:106B900002D0E82EFCD79E96C69E26C5C9FFFF0EE2
:106BA0009EB602D0E82EFCD79E96C69E25C5C9FF8C
:106BB000FF0E9EB602D0E82EFCD79E96C69EC95206
:106BC000FF0E9EB602D0E82EFCD7898A0F01C9506D
:106BD000FF0AD8A407EF37F00501FE0E376F15A4A2
:106BE000379901EC31F0AFC538F5B0C539F5B1C50D
:106BF0003AF5B2C53BF5B3C53CF5B4C53DF5B5C5F1
:106C00003EF50784BAC166F1BBC167F1BCC168F14A
:106C1000BDC169F14BC14FF14CC150F14DC151F1B2
:106C20004EC152F157C159F158C15AF100011650E5
:106C3000010AD8B42AEF36F000011650020AD8B47F
:106C400040EF36F000011650040AD8B456EF36F083
:106C500007EF37F08BA0379B5FEC22F000C1DAF131
:106C600001C1DBF102C1DCF103C1DDF100C13FF57F
:106C700001C140F502C141F503C142F575EF36F09F
:106C80005FEC22F000C1DAF101C1DBF102C1DCF1FD
:106C900003C1DDF15CEC23F000C147F501C148F50B
:106CA00002C149F503C14AF507EF37F0379BDAC156
:106CB0003FF5DBC140F5DCC141F5DDC142F55FECDC
:106CC00022F000C14BF501C14CF502C14DF503C1E5
:106CD0004EF55CEC23F000C14FF501C150F502C147
:106CE00051F503C152F575EF36F00501616780EF8C
:106CF00036F0626780EF36F0636780EF36F06467E6
:106D000084EF36F099EF36F0DAC100F1DBC101F122
:106D1000DCC102F1DDC103F161C504F162C505F119
:106D200063C506F164C507F165EC2FF003BF07EFFB
:106D300037F059C143F55AC144F5B9C545F50501C8
:106D4000110E326F899A400EC76E200EC66E9E9647
:106D5000C69E060EC96EFF0E9EB602D0E82EFCD768
:106D6000898A899A9E96C69E020EC96EFF0E9EB6AD
:106D700002D0E82EFCD79E96C69E27C5C9FFFF0EFF
:106D80009EB602D0E82EFCD79E96C69E26C5C9FFA9
:106D9000FF0E9EB602D0E82EFCD79E96C69E25C555
:106DA000C9FFFF0E9EB602D0E82EFCD725EE37F0C5
:106DB000322F02D0E7EF36F09E96C69EDECFC9FF97
:106DC000FF0E9EB602D0E82EFCD7D8EF36F0898AA7
:106DD000899A9E96C69E050EC96EFF0E9EB602D07B
:106DE000E82EFCD79E96C69EC952FF0E9EB602D0D4
:106DF000E82EFCD7C9B0F2EF36F0898A0501100EF3
:106E00002527E86A2623E86A2723E86A28231590BD
:106E10000794120021C500F122C501F123C502F13A
:106E200024C503F1899A400EC76E200EC66E9E9649
:106E3000C69E0B0EC96EFF0E9EB602D0E82EFCD782
:106E40009E96C69E02C1C9FFFF0E9EB602D0E82ED6
:106E5000FCD79E96C69E01C1C9FFFF0E9EB602D00A
:106E6000E82EFCD79E96C69E00C1C9FFFF0E9EB6B7
:106E700002D0E82EFCD79E96C69EC952FF0E9EB643
:106E800002D0E82EFCD725EE37F00501100E326F48
:106E90009E96C69EC952FF0E9EB602D0E82EFCD723
:106EA000C9CFDEFF322F48EF37F0898A1200899A66
:106EB000400EC76E200EC66E9E96C69E900EC96E80
:106EC000FF0E9EB602D0E82EFCD79E96C69E000E00
:106ED000C96EFF0E9EB602D0E82EFCD79E96C69EC7
:106EE000000EC96EFF0E9EB602D0E82EFCD79E960D
:106EF000C69E000EC96EFF0E9EB602D0E82EFCD7CD
:106F00009E96C69EC952FF0E9EB602D0E82EFCD7B2
:106F1000C9CF2DF59E96C69EC952FF0E9EB602D0D1
:106F2000E82EFCD7C9CF2EF5898A120001EC31F08A
:106F300005012F51020A16E005012F51030A19E03D
:106F400005012F51040A24E005012F51050A2BE009
:106F500005012F51060A39E005012F51070A3FE0CC
:106F6000F7EF37F0602FF5EF37F05FC560F5F7EF1B
:106F700037F0B0C500F101010F0E001701010051FB
:106F8000000A35E001010051050A31E0F5EF37F064
:106F9000B0C500F101010F0E001701010051000AF8
:106FA00026E0F5EF37F00501B051000A20E00501B9
:106FB000B051150A1CE00501B051300A18E0050176
:106FC000B051450A14E0F5EF37F00501B051000A61
:106FD0000EE00501B051300A0AE0F5EF37F0050187
:106FE000B051000A04E0F5EF37F01590120015805B
:106FF00012008B9031EC2EF0B9C5E8FFD70802E300
:1070000031EC2EF0B9C5E8FFC80802E331EC2EF0F0
:10701000B9C5E8FFB90802E331EC2EF0B9C5E8FFC5
:10702000AA0802E331EC2EF0B9C5E8FF9B0802E3A1
:1070300031EC2EF08DEC35F0F29CF29E8B94C69ADA
:10704000C2909482948C720ED36ED3A4FED789968C
:107050008A909390F29AF2949D909E909D929E9227
:10706000F298F292A7EC32F0FF0EE8CF00F0E82E93
:10707000FED7002EFCD7F290F286815081A843EF14
:1070800038F0F29E0300700ED36EF296F2901584E3
:0A709000038052EC2EF099EF0BF094
:10BF0000E844F926000C160C2B0C3F0C520C640C68
:10BF1000760C860C960CA50CB30CC10CCF0CDC0C6B
:06BF2000E80CF40C000C1B
:0200000400F00A
:0100C800FE39
:00000001FF
